:020000040000FA
:0400000007EF00F016
:1000080075822FED42F08BEF4AF066C0D9FF67C0CA
:10001800DAFFDE6ADD6A68C00BF039EC45F00BC028
:10002800B6F00CC0B7F00001B7BF0B0CD890B635CE
:10003800D96EB735DA6E940ED926010EDA22DECFE4
:10004800D0F0DDCFD1F0D051D11101E10C0C66C058
:10005800D9FF67C0DAFFD0C0DEFFD1C0DDFFD0C056
:10006800D9FFD1C0DAFFDF5012E020EE01F0D05105
:10007800D926D151DA22DF5008EC57F00001C26FBF
:10008800C2B105D06950D8A4C2A5000C0A0CD0C0D2
:10009800D9FFD1C0DAFFDF6A20EE01F0D051D926AE
:1000A800D151DA22B6C0DFFF20EE01F0D051D926B7
:1000B800D151DA22DF50B7EC40F00001C26FC2B173
:1000C800030C695002E0C2B50A0CC96BCA6BCB6B52
:1000D800CC6BD0C044F0D1C045F0466A476A486A44
:1000E800496A3CEC38F00001CF6FCF0501E0D4D06D
:1000F800CD6BCE6BCE5105E1040ECD5D01E390D002
:1001080001D08ED0CDC080F0CEC081F0803B813B45
:10011800F00E811780510F0B8113F00E8017D0C09D
:1001280082F0D1C083F08051822781518323EC0E65
:100138008225C36F010E8321C46F20EE04F0C351E2
:10014800D926C451DA22DF5005E1A86BA96BAA6B46
:10015800AB6B55D020EE09F0C351D926C451DA2231
:10016800DF50816F806B20EE0AF0C351D926C4514D
:10017800DA22DF50826F82C083F0846B856B866BD6
:1001880084C086F083C085F0846B836B20EE0BF00F
:10019800C351D926C451DA22DF50876F87C088F04F
:1001A800896B8A6B8B6B88C08BF08A6B896B886BC9
:1001B800835188118C6F845189118D6F85518A11F3
:1001C8008E6F86518B118F6F80518C11906F81517A
:1001D8008D11916F000E8E11926F000E8F11936F1B
:1001E80020EE08F0C351D926C451DA22DF5090110D
:1001F800A86F9151A96F9251AA6F9351AB6FCD51CE
:10020800040DF350980FD96EDA6AA8C0DEFFA9C0B2
:10021800DEFFAAC0DEFFABC0DEFFCD4BCE2B6AD718
:10022800CD6BCE6BCD51CE1103E0CD07D8A0CE0754
:10023800CD51040DF350980FD96EDA6ADECFC9F0AC
:10024800DECFCAF0DECFCBF0DECFCCF0C951CA1179
:10025800CB11CC1105E1000EAD6F020EAC6F11D0C1
:10026800D0C044F0D1C045F0C9C046F0CAC047F07C
:10027800CBC048F0CCC049F03CEC38F00001AC6F82
:10028800AD6BACC0CFF0CF5107E0CD4BCE2BCE51EC
:1002980003E1040ECD5DCCE3030ECF1901E1010C9F
:1002A800CF5101E00D0C20EE3AF0D051D926D151B2
:1002B800DA22DF50816F806B20EE39F0D051D926D9
:1002C800D151DA22DF508013020E8119801101E02A
:1002D8000D0C20EE45F0D051D926D151DA22DF504D
:1002E800816F806B20EE44F0D051D926D151DA22AB
:1002F800DF50801380C0C5F081C0C6F0C76BC86BE3
:10030800C551C611C711C81155E120EE53F0D0519F
:10031800D926D151DA22DF50816F806B20EE54F05C
:10032800D051D926D151DA22DF50826F82C083F0B2
:10033800846B856B866B84C086F083C085F0846B84
:10034800836B20EE55F0D051D926D151DA22DF50F7
:10035800876F87C088F0896B8A6B8B6B88C08BF03E
:100368008A6B896B886B835188118C6F84518911D2
:100378008D6F85518A118E6F86518B118F6F8051C9
:100388008C11906F81518D11916F000E8E11926FAB
:10039800000E8F11936F20EE52F0D051D926D15113
:1003A800DA22DF509011C56F9151C66F9251C76F15
:1003B8009351C86F20EE16F0D051D926D151DA22C8
:1003C800C5C0DEFFC6C0DEFFC7C0DEFFC8C0DEFF97
:1003D80020EE3EF0D051D926D151DA2210EE03F0AA
:1003E800D051E126D151E222DFCFE7FF20EE03F022
:1003F800D051D926D151DA22DE040AE020EE03F0EA
:10040800D051D926D151DA22020EDE1801E00D0CA6
:10041800C5C00BF0C6C00CF0C7C00DF0C8C00EF0C8
:1004280020EE03F0D051D926D151DA22DF500F6ED9
:10043800106A116A126A49EC4FF00BC0C5F00CC083
:10044800C6F00DC0C7F00EC0C8F020EE3BF0D0518A
:10045800D926D151DA2210EE02F0D051E126D1513D
:10046800E222DFCFE7FF20EE02F0D051D926D151AA
:10047800DA22DF50D8B40D0C20EE02F0D051D92684
:10048800D151DA22DF50806F20EE02F0D051D92608
:10049800D151DA22DF50816F8105801501E00D0C02
:1004A80020EE40F0D051D926D151DA22DF50816FA9
:1004B800806B20EE3FF0D051D926D151DA22DF509F
:1004C800801320EE08F0D051D926D151DA2280C00D
:1004D800DEFF81C0DDFF20EE08F0D051D926D151D2
:1004E800DA22DF50806F0F0E801701E00D0C20EE2E
:1004F80042F0D051D926D151DA22DF50816F806B7A
:1005080020EE41F0D051D926D151DA22DF508013A4
:1005180080C0BAF081C0BBF0BC6BBD6BBA51BB11D7
:10052800BC11BD1155E120EE4FF0D051D926D15163
:10053800DA22DF50816F806B20EE50F0D051D9263F
:10054800D151DA22DF50826F82C083F0846B856BD1
:10055800866B84C086F083C085F0846B836B20EE45
:1005680051F0D051D926D151DA22DF50876F87C098
:1005780088F0896B8A6B8B6B88C08BF08A6B896B70
:10058800886B835188118C6F845189118D6F8551C7
:100598008A118E6F86518B118F6F80518C11906FDD
:1005A80081518D11916F000E8E11926F000E8F1177
:1005B800936F20EE4EF0D051D926D151DA22DF5078
:1005C8009011BA6F9151BB6F9251BC6F9351BD6F2F
:1005D80020EE3CF0D051D926D151DA22DF50806F7D
:1005E80020EE3DF0D051D926D151DA22DF50816F6B
:1005F8008051B86F81C0B9F0B851B91101E10D0C43
:1006080020EE08F0D051D926D151DA22DECF80F081
:10061800DDCF81F0040E826FD89081338033822F32
:10062800FBD7B8518025836FB9518121846F856BC1
:10063800D8B0852B866BC5518325B26FC6518421EE
:10064800B36FC7518521B46FC8518621B56FB251B8
:10065800BA5DB351BB59B451BC59B551BD5901E24A
:100668000D0CB251BA5D0B6EB351BB590C6EB4513F
:10067800BC590D6EB551BD590E6E20EE02F0D05129
:10068800D926D151DA22DF500F6E106A116A126A28
:100698000BEC50F00BC0BEF00CC0BFF00DC0C0F0AA
:1006A8000EC0C1F00001BE51BF11C011C11101E15E
:1006B8000D0C010ECF6FC151C01105E1F60EBE5DE4
:1006C8000F0EBF5902E3020ECF6FC151C01105E1F1
:1006D800F60EBE5DFF0EBF5902E3030ECF6F020E8A
:1006E800BE25806F000EBF21816F000EC021826F72
:1006F800000EC121836F20EE12F0D051D926D151BE
:10070800DA2280C0DEFF81C0DEFF82C0DEFF83C048
:10071800DEFF20EE1AF0D051D926D151DA22C9C015
:10072800DEFFCAC0DEFFCBC0DEFFCCC0DEFFB851A3
:10073800C925806FB951CA21816F000ECB21826F04
:10074800000ECC21836F20EE1EF0D051D926D15156
:10075800DA2280C0DEFF81C0DEFF82C0DEFF83C0F8
:10076800DEFFB251C925806FB351CA21816FB451E0
:10077800CB21826FB551CC21836F20EE26F0D0516A
:10078800D926D151DA2280C0DEFF81C0DEFF82C0C7
:10079800DEFF83C0DEFF030ECF1901E08CD020EE10
:1007A80008F0D051D926D151DA22DE50DE1001E00E
:1007B8000D0C20EE5BF0D051D926D151DA22DF5052
:1007C800816F806B20EE5CF0D051D926D151DA22AE
:1007D800DF50826F82C083F0846B856B866B84C028
:1007E80086F083C085F0846B836B20EE5DF0D0517A
:1007F800D926D151DA22DF50876F87C088F0896BFC
:100808008A6B8B6B88C08BF08A6B896B886B835182
:1008180088118C6F845189118D6F85518A118E6F63
:1008280086518B118F6F80518C11906F81518D1172
:10083800916F000E8E11926F000E8F11936F20EE44
:100848005AF0D051D926D151DA22DF509011946F45
:100858009151956F9251966F9351976F20EE22F0B8
:10086800D051D926D151DA2294C0DEFF95C0DEFFDF
:1008780096C0DEFF97C0DEFF20EE12F0D051D926D9
:10088800D151DA22DECF80F0DECF81F0DECF82F0E8
:10089800DECF83F0020ED8908037813782378337D6
:1008A800E82EF9D780C0AEF081C0AFF082C0B0F0BA
:1008B80083C0B1F0B7D020EE08F0D051D926D1517D
:1008C800DA22DE50DE1001E10D0C20EE1EF0D051D0
:1008D800D926D151DA22DECF80F0DECF81F0DECF0B
:1008E80082F0DECF83F0C5518025846FC651812107
:1008F800856FC7518221866FC8518321876F20EE8B
:1009080022F0D051D926D151DA2284C0DEFF85C029
:10091800DEFF86C0DEFF87C0DEFF020ECF196BE068
:1009280020EE12F0D051D926D151DA22DECF80F054
:10093800DECF81F0DECF82F0DECF83F0010E8015AE
:10094800846F856B866B876B20EE12F0D051D926A9
:10095800D151DA22DECF88F0DECF89F0DECF8AF0FF
:10096800DECF8BF0030E8803F3CF8CF0F4CF8DF03D
:100978008E6B8F6B8903F3508D27F4508E23000EF6
:100988008F238803F3508D27F4508E23000E8F2376
:10099800030E8A03F3508E27F4508F23000E890329
:1009A800F3508E27F4508F23000E8803F3508E27C0
:1009B800F4508F23030E8B03F3508F27000E8A0306
:1009C800F3508F27000E8903F3508F27000E8803FA
:1009D800F3508F27D8908F338E338D338C338451D7
:1009E8008C25AE6F85518D21AF6F86518E21B06FEA
:1009F80087518F2116D020EE12F0D051D926D1512F
:100A0800DA22DECF80F0DECF81F0DECF82F0DECFDB
:100A180083F0D8908035AE6F8135AF6F8235B06F77
:100A28008335B16FFF0EAE25806F010EAF21816F48
:100A3800000EB021826F000EB121836F0A0E05D01F
:100A4800D8908333823381338033E82EF9D720EE70
:100A580016F0D051D926D151DA228051DE5C81516D
:100A6800DE588251DE588351DE5801E20D0C20EE2B
:100A78000EF0D051D926D151DA22DE68DE68DE6860
:100A8800DD68DD52DD5210EE0AF0D051E126D15179
:100A9800E222DECFE6FFDECFE6FFDECFE6FFDECFE7
:100AA800E6FF20EE05F0D051D926D151DA22800E8A
:100AB800DF6E030ECF1901E0D3D120EE5FF0D051E5
:100AC800D926D151DA22DF50816F806B20EE5EF09B
:100AD800D051D926D151DA22DF50801380058111F7
:100AE80001E0BED1D0C039F0D1C03AF0C9293B6E7F
:100AF800000ECA213C6E000ECB213D6E000ECC21AB
:100B08003E6E06EC4DF0000901E0AAD1000120EE8E
:100B180005F0D051D926D151DA22DF6A22EE2DF024
:100B2800D051D926D151DA22DF50816F806B22EE65
:100B38002CF0D051D926D151DA22DF508013550E2E
:100B4800801903E1AA0E8119D8A48AD120EE2FF0CA
:100B5800D051D926D151DA22DF50816F806B20EE37
:100B680030F0D051D926D151DA22DF50826F82C0BD
:100B780083F0846B856B866B84C086F083C085F0B8
:100B8800846B836B20EE31F0D051D926D151DA2213
:100B9800DF50876F87C088F0896B8A6B8B6B88C042
:100BA8008BF08A6B896B886B835188118C6F8451A9
:100BB80089118D6F85518A118E6F86518B118F6FB8
:100BC80080518C11906F81518D11916F000E8E1193
:100BD800926F000E8F11936F20EE2EF0D051D92610
:100BE800D151DA22DF509011946F9151956F925143
:100BF800966F9351976F520E941909E1520E9519F9
:100C080006E1610E961903E1410E9719D8A428D17F
:100C180022EE13F0D051D926D151DA22DF50816F5C
:100C2800806B22EE14F0D051D926D151DA22DF5050
:100C3800826F82C083F0846B856B866B84C086F07C
:100C480083C085F0846B836B22EE15F0D051D926D2
:100C5800D151DA22DF50876F87C088F0896B8A6BA1
:100C68008B6B88C08BF08A6B896B886B835188117A
:100C78008C6F845189118D6F85518A118E6F8651C1
:100C88008B118F6F80518C11906F81518D11916FE5
:100C9800000E8E11926F000E8F11936F22EE12F0DC
:100CA800D051D926D151DA22DF509011946F915149
:100CB800956F9251966F9351976F720E941909E13F
:100CC800720E951906E1410E961903E1610E971906
:100CD800D8A4C6D022EE17F0D051D926D151DA22A5
:100CE800DF50816F806B22EE18F0D051D926D15198
:100CF800DA22DF50826F82C083F0846B856B866B4B
:100D080084C086F083C085F0846B836B22EE19F073
:100D1800D051D926D151DA22DF50876F87C088F0A9
:100D2800896B8A6B8B6B88C08BF08A6B896B886B3D
:100D3800835188118C6F845189118D6F85518A1167
:100D48008E6F86518B118F6F80518C11906F8151EE
:100D58008D11916F000E8E11926F000E8F11936F8F
:100D680022EE16F0D051D926D151DA22DF50901157
:100D7800946F9151956F9251966F9351976F20EEA2
:100D88000EF0D051D926D151DA2294C0DEFF95C099
:100D9800DEFF96C0DEFF97C0DEFF22EE1BF0D051CB
:100DA800D926D151DA22DF50816F806B22EE1CF0F8
:100DB800D051D926D151DA22DF50826F82C083F018
:100DC800846B856B866B84C086F083C085F0846BEA
:100DD800836B22EE1DF0D051D926D151DA22DF5093
:100DE800876F87C088F0896B8A6B8B6B88C08BF0A4
:100DF8008A6B896B886B835188118C6F8451891138
:100E08008D6F85518A118E6F86518B118F6F80512E
:100E18008C11906F81518D11916F000E8E11926F10
:100E2800000E8F11936F22EE1AF0D051D926D151AE
:100E3800DA22DF509011946F9151956F9251966F0D
:100E48009351976F20EE0AF0D051D926D151DA226A
:100E580094C0DEFF95C0DEFF96C0DEFF97C0DEFFC0
:100E6800D0C0D9FFD1C0DAFFCFC0DFFF0101924B5C
:100E7800932B000120EE06F0D051D926D151DA2269
:100E880092C1DEFF93C1DDFF000C0C6A0B6ABDEC5A
:100E980056F00F0B0101F86F9F6B070E966E010E4F
:100EA800F96FAB6B0F0EC16E926893689468948E5D
:100EB800929092928982020EF76F0CEC56F09294FF
:100EC800898492988998929E899E956893682C0E39
:100ED8000001806FFB0E816FA90E826FFF0E836F7A
:100EE800F00E846FFE0E856F310E866FFF0E876FD2
:100EF800D3EC56F0A4EC56F017D0A30E0001806F87
:100F0800FE0E816F82CF82F0836BD3EC56F0150E04
:100F18000101DA6F4B0ED96FBE0EE82EFED7D92F1E
:100F2800FCD7DA2FFAD700F082B2E7D7DDEC46F02B
:100F38000101F86F4E0E0001806FFC0E816FF8C141
:100F480082F0836BD3EC56F00400150E0101DA6FC2
:100F58004B0ED96FBE0EE82EFED7D92FFCD7DA2F4D
:100F6800FAD700F0CD929D90CF0ECD16CD8ECD80C4
:100F7800F286F180F288F19CF28E96EC52F089921A
:100F880089944CEC49F04CEC49F0000E0B6E340E91
:100F9800B0EC53F04C0E0F6EFF0E106ECEEC4FF00F
:100FA800A90E0F6EFF0E106ECEEC4FF0000E0B6EFA
:100FB800390EB0EC53F089800400C0EC34F04CECEE
:100FC8003BF0F0EC4AF0000E0B6E800EB0EC53F0E4
:100FD8000101F8510F0D340EF3240F6E0C0EF4209E
:100FE800106ECEEC4FF00101AA5101E1F2D0910E42
:100FF8000001806FFD0E816FD3EC56F0EDEC50F0E0
:101008000FC0E9F110C0EAF111C0EBF112C0ECF128
:101018000101E951EA11EB11EC1117E1950E0001FC
:10102800806FFC0E816FE9C182F0EAC183F0EBC1E9
:1010380084F0ECC185F0D3EC56F00A0E0E6E000E6B
:101048000F6A106A116A14EC53F00101ED6BEE6B34
:10105800EEBF05D0EE5119E1040EED5D16E2D90E92
:101068000001806FFF0E816FE90E0101ED25D96E39
:10107800010EEE21DA6EDF500001826F836BD3EC34
:1010880056F00101ED4BEE2BE3D7590E0001806FAE
:10109800FB0E816FD3EC56F01B0E0001806FFC0E27
:1010A800816FD3EC56F022EE08F000EECAF01F0E66
:1010B800DBCFEBFFE806FCE2D10E0001EA6FFF0E82
:1010C800EB6FFDEC35F0CAC084F1CBC085F1CCC024
:1010D80086F1CDC087F101018451851186118711F0
:1010E80078E0010E0001806FFC0E816F84C182F0F0
:1010F80085C183F086C184F087C185F0D3EC56F0B2
:10110800080E0001A36F020EA46F84C1DAF185C135
:10111800DBF186C1DCF10101D96B000ED925000194
:10112800A56F010E0101DA210001A66F000E010171
:10113800DB210001A76F000E0101DC210001A86F6F
:1011480077EC0EF0080E626E020E636E340E646E5B
:101158000A0E656E676A080E666EE70E686E010E07
:10116800696E61EC11F00101EF6BF06BF0BF05D017
:10117800F05119E1080EEF5D16E2D50E0001806FFF
:10118800FF0E816F340E0101EF25D96E0A0EF02192
:10119800DA6EDF500001826F836BD3EC56F00101E9
:1011A800EF4BF02BE3D72AEE34F0DF50DD6FDE6B28
:1011B800DF6BE06B790E0001806FFE0E816FDDC181
:1011C80082F0DEC183F0DFC184F0E0C185F0D3ECAA
:1011D80056F00101ABAF13D0946889928982150E3D
:1011E8000101DA6F4B0ED96FBE0EE82EFED7D92F4C
:1011F800FCD7DA2FFAD700F030EC3EF0EED7F951F1
:101208000CE0B10E0001806FFD0E816FD3EC56F03B
:10121800020E0101A36F220E0BD0A10E0001806FF8
:10122800FD0E816FD3EC56F0010E0101A36F040E81
:10123800A26FE36BE46BF16B899E000EF36F010EF6
:10124800F26FF3BF05D0F35168E1040EF25D65E279
:101258000F0EF203F3CFD9F1F4CFDAF1F303F35021
:10126800DA27240ED9250B6E0D0EDA210C6E38EC18
:1012780054F00C5003E1030E0B5C4BE3100E00011D
:10128800806FFE0E816F0F0E0101F203F3CFD9F1CB
:10129800F4CFDAF1F303F350DA27240ED92500014D
:1012A800826F0D0E0101DA210001836FD3EC56F035
:1012B800F2C1D9F1F3C1DAF1050ED8900101D9379D
:1012C800DA37E82EFAD7080ED9250001D26F020EB8
:1012D8000101DA210001D36F0F0E0101F203F3CFF0
:1012E800DBF1F4CFDCF1F303F350DC27240EDB252C
:1012F8000001D46F0D0E0101DC210001D56F030E32
:10130800D66FA1EC16F00101E56FE66BE5513DECF7
:1013180053F00101F24BF32B94D7899E000E0B6E0C
:10132800C00EB0EC53F05CEC56F0000E0B6EC00E25
:10133800B0EC53F0910E0F6EFF0E106ECEEC4FF026
:10134800F8D081A893940EEC57F00B500101E26F8E
:10135800E25101E1CFD0F1C1E1F1F40E0B6E010EC3
:101368000C6EC0EC4EF00101F16FF4B9F19F3A0E2A
:101378000001806FFF0E816FF1C182F0836B010164
:10138800010EF4A9000E0001846F856BD3EC56F0B2
:101398000101F4A91DD0600EF1191AE15F0EE119DF
:1013A80017E1F7832AEE34F0A3C1DFFF2AEE35F008
:1013B800A2C1DFFF89845B6A020E5A6E3DEC3DF0E4
:1013C8008994F793726A7CEC56F00101F16BB1D005
:1013D800F95144E0F451100B0001C96F000ECA6FB7
:1013E8000101F1511EEC3FF0C9C0F5F1CAC0F6F198
:1013F800080E0101F519F61101E100F0070E0101CF
:10140800F519F61102E185EC51F00101F505F61127
:1014180002E1B3EC4BF0020EF519F61102E14AECC9
:101428003CF0030EF519F61106E149EC2FF0E1C086
:10143800E3F1E2C0E4F1050E0101F519F61106E148
:101448004EEC3AF0EAC0E3F1EBC0E4F1090E010119
:10145800F519F6114CE162EC4CF049D0F451100B3F
:101468005A6E000E5B6EF151ADEC1DF05AC0F5F1ED
:101478005BC0F6F1070E0101F519F61102E121EC46
:1014880051F0020EF519F61102E18BEC53F0F50557
:10149800F61102E161EC1BF0030EF519F61102E1F9
:1014A800B9EC50F0040EF519F61102E19EEC55F076
:1014B800050EF519F61102E1CBEC45F0060E010117
:1014C800F519F61102E117EC57F0080EF519F611A7
:1014D80002E12BEC37F0090EF519F61102E15EEC8A
:1014E80048F00A0EF519F61102E1E0EC47F00101A7
:1014F800A46B1FD0DDEC46F001019F6FA05119E0ED
:10150800F8519F1916E0898E000E0B6EC00EB0ECD4
:1015180053F05CEC56F0000E0B6EC00EB0EC53F0BE
:10152800FC0E0F6EFE0E106ECEEC4FF09FC1F8F160
:1015380032D082B230D0050E0101E319E4112BE05C
:1015480000D7A30E0001806FFE0E816F82CF82F05C
:10155800836BD3EC56F0150E0101DA6F4B0ED96F81
:10156800BE0EE82EFED7D92FFCD7DA2FFAD700F017
:101578000400000E0B6EC00EB0EC53F05CEC56F09D
:10158800000E0B6EC00EB0EC53F0540E0F6EFF0E33
:10159800106ECEEC4FF082B2D4D7150E0101DA6F7F
:1015A8004B0ED96FBE0EE82EFED7D92FFCD7DA2FF7
:1015B800FAD700F0000E08EC57F001019E6FDA0E22
:1015C8000001806FFC0E816F9EC182F0836BD3ECAB
:1015D80056F0150E0101DA6F4B0ED96FBE0EE82ECC
:1015E800FED7D92FFCD7DA2FFAD700F08994899241
:1015F8000001D26BD36B5B0ED46FFB0ED56FD66B2D
:1016080054EC4DF0D9D4A5C0B8F0A6C0B9F0A9C023
:10161800D9FFAAC0DAFFDE6ADD6AA3C00CF0A4C055
:101628000DF079EC4EF00001B76FB75102E0B751F9
:10163800120020EE05F0A351D926A451DA22DF507A
:1016480008E020EE05F0A351D926A451DA22DF5094
:10165800120020EE04F0A351D926A451DA22DFA209
:10166800070C20EE06F0A351D926A451DA2210EE79
:1016780006F0A351E126A451E222E6CFAFF0E6CF6F
:10168800B0F0E6CFB1F0E6CFB2F0A751AF25B36F17
:10169800A851B021B46F000EB121B56F000EB22170
:1016A800B66FDE50B35DDE50B459DE50B559DE502A
:1016B800B65901E3E2D2A76BA86BDFD220EE06F0A1
:1016C800A351D926A451DA22FF0EDE14AB6F010E06
:1016D800DE14AC6F000EDE14AD6F000EDE14AE6FBC
:1016E800AB51AC11AD11AE1101E032D220EE06F0D3
:1016F800A351D926A451DA22DECFABF0DECFACF06D
:10170800DECFADF0DECFAEF00A0E05D0D890AE3306
:10171800AD33AC33AB33E82EF9D7A3C0D9FFA4C09F
:10172800DAFF10EE02F0DE50E126DD50E222E7504B
:10173800AF6FAF05AB15BA6FBA5101E099D020EE83
:1017480006F0A351D926A451DA22DE50DE10DE10AD
:10175800DE1022E120EE0EF0A351D926A451DA22A0
:10176800DECFC1F0DECFC2F0DECFC3F0DECFC4F0F3
:10177800C151C211C311C4112FE1A3C0D9FFA4C024
:10178800DAFFDECF8CF0DDCF8DF08E6B8F6B906B38
:10179800916B16EC32F018D0A3C0D9FFA4C0DAFFC1
:1017A800DECF8CF0DDCF8DF020EE12F0A351D926DC
:1017B800A451DA22DECF8EF0DECF8FF0DECF90F0AC
:1017C800DECF91F016EC32F08CC0C1F08DC0C2F0C3
:1017D8008EC0C3F08FC0C4F0C151C211C311C4116F
:1017E80001E14FD2C105C211C311C41109E120EEB4
:1017F80005F0A351D926A451DA22020EDF6E020C9D
:10180800C1290FE1C2290DE1C3290BE1C42909E16E
:1018180020EE05F0A351D926A451DA22010EDF6E7D
:10182800010C20EE12F0A351D926A451DA22C1C02E
:10183800DEFFC2C0DEFFC3C0DEFFC4C0DEFF20EE95
:101848000EF0A351D926A451DA22DE50DE10DE10A4
:10185800DE100EE120EE0EF0A351D926A451DA22B3
:10186800C1C0DEFFC2C0DEFFC3C0DEFFC4C0DEFFF2
:1018780020EE16F0A351D926A451DA22A3C0E1FF25
:10188800A4C0E2FF00EE2AF0E650E926E550EA227D
:10189800DE50EE1816E1DE50EE1813E1DE50EE18B9
:1018A80010E1DE50EE180DE1A3C0D9FFA4C0DAFFA5
:1018B800DECF24F0DDCF25F0D4EC42F0000901E0C2
:1018C80083D1A3C0D9FFA4C0DAFFDECF0BF0DDCFF0
:1018D8000CF0000120EE12F0A351D926A451DA220F
:1018E800DECF0DF0DECF0EF0DECF0FF0DECF10F042
:1018F80056EC46F00BC0BDF00CC0BEF00DC0BFF0FA
:101908000EC0C0F00001BD51BE11BF11C01101E1F0
:101918006ED7BA51BD27000EBE23BF23C023A7C070
:10192800ABF0A8C0ACF0090EAD6FD890AC33AB33B8
:10193800AD2FFBD7ABC0BBF0ACC0BCF0BB51BC11EA
:1019480001E1C3D0BA51BB25AB6F000EBC21AC6F0F
:10195800A3C0D9FFA4C0DAFF10EE02F0DE50E126E2
:10196800DD50E222E750AD6FAE6BAB51AD5DAC51CF
:10197800AE5912E2A3C0D9FFA4C0DAFF10EE02F0FC
:10198800DE50E126DD50E222E750AB6FBA51AB5D85
:10199800BB6FBC6BD8A0BC07B8C01AF0B9C01BF0AD
:1019A800BDC01CF0BEC01DF0BFC01EF0C0C01FF0FF
:1019B800BBC020F0BCC021F0A3C0D9FFA4C0DAFF8F
:1019C80010EE01F0DE50E126DD50E222E750DAECBD
:1019D80048F0000901E0F8D00001BB51AB6FBC51E1
:1019E800AC6FAD6BAE6BA3C0D9FFA4C0DAFF10EE2D
:1019F8002AF0DE50E126DD50E222E6CFAFF0E6CF56
:101A0800B0F0E6CFB1F0E6CFB2F0BD51AF5DB36F45
:101A1800BE51B059B46FBF51B159B56FC051B25929
:101A2800B66FAB51B35DAC51B459AD51B559AE5168
:101A3800B6593CE2A3C0D9FFA4C0DAFFDECFABF0B1
:101A4800DDCFACF02E0EAB250B6E000EAC210C6E6C
:101A5800A3C0D9FFA4C0DAFF10EE2AF0DE50E126B9
:101A6800DD50E222E6CFADF0E5CFAEF0BD51AD5F7F
:101A7800BE51AE5B090ED890AD37AE37E82EFBD716
:101A8800AD51B8250D6EAE51B9210E6E020E106E15
:101A98000F6A59EC54F0A3C0D9FFA4C0DAFF10EEC6
:101AA80004F0DE50E126DD50E222E76ABBC0ABF06D
:101AB800BCC0ACF0090ED890AB37AC37E82EFBD7DA
:101AC800ABC0C5F0ACC0C6F0BBD020EE0AF0A35145
:101AD800D926A451DA2210EE06F0A351E126A4512A
:101AE800E222DE50E65CDE50E658DE50E658DE5074
:101AF800E6581FE3A3C0D9FFA4C0DAFFDECF24F065
:101B0800DDCF25F0D4EC42F0000901E05DD0A3C0A0
:101B1800D9FFA4C0DAFF10EE2AF0DE50E126DD502E
:101B2800E222BDC0E6FFBEC0E6FFBFC0E6FFC0C000
:101B3800E6FF000120EE16F0A351D926A451DA22BF
:101B4800BDC0DEFFBEC0DEFFBFC0DEFFC0C0DEFF1F
:101B5800AB69010EAC6F20EE06F0A351D926A45153
:101B6800DA22DECFADF0DDCFAEF0AB51AD17AC5120
:101B7800AE17AD510008C56FAE51D8A0E82A0208CB
:101B8800C66FC551A75DC651A85904E2A7C0C5F0E4
:101B9800A8C0C6F0A3C0D9FFA4C0DAFFDECF39F0D1
:101BA800DDCF3AF020EE16F0A351D926A451DA225F
:101BB800DECF3BF0DECF3CF0DECF3DF0DECF3EF0B7
:101BC80006EC4DF0000902E0000122D60001AB69E5
:101BD800010EAC6F20EE06F0A351D926A451DA22EB
:101BE800DECFADF0DDCFAEF0AB51AD17AC51AE17D7
:101BF800A3C0D9FFA4C0DAFFDECFAFF0DDCFB0F0CD
:101C0800AD51AF27AE51B0232E0EAF250B6E000E8F
:101C1800B0210C6EB8C00DF0B9C00EF0C5C00FF001
:101C2800C6C010F059EC54F0A3C0D9FFA4C0DAFF25
:101C380010EE04F0DE50E126DD50E222010EE76EE0
:101C4800C551B827C651B92320EE06F0A351D926AD
:101C5800A451DA22C551DE26C651DE22000EDE224C
:101C6800DE22A9C0D9FFAAC0DAFFC551DE26C651B7
:101C7800DD22C551A75FC651A85BA751A81101E095
:101C88001DD520EE06F0A351D926A451DA2210EE74
:101C98000AF0A351E126A451E222DE50E65CDE50B0
:101CA800E658DE50E658DE50E65814E220EE06F01C
:101CB800A351D926A451DA2210EE0AF0A351E12645
:101CC800A451E222DECFE6FFDECFE6FFDECFE6FF5D
:101CD800DECFE6FF20EE04F0A351D926A451DA2284
:101CE800000EDB8A000CA3C00CF0A4C00DF079EC48
:101CF8004EF00001BD6FBD5102E0BD51120020EE53
:101D080005F0A351D926A451DA22DF5008E020EECD
:101D180005F0A351D926A451DA22DF50120020EE93
:101D28000AF0A351D926A451DA22A551DE5CA651A6
:101D3800DE58A751DE58A851DE5816E220EE04F00E
:101D4800A351D926A451DA22DFB20ED020EE0AF030
:101D5800A351D926A451DA22DECFA5F0DECFA6F012
:101D6800DECFA7F0DECFA8F020EE06F0A351D926EB
:101D7800A451DA22DECFB9F0DECFBAF0DECFBBF065
:101D8800DECFBCF0BE6BBF6BC06BC16B20EE06F044
:101D9800A351D926A451DA22BEC0DEFFBFC0DEFFA0
:101DA800C0C0DEFFC1C0DEFFA551A611A711A81152
:101DB80001E119D2A3C0D9FFA4C0DAFF10EE02F0E6
:101DC800DE50E126DD50E222E750A96FA9C0AAF053
:101DD800AB6BAC6BAD6B090ED890AA37AB37AC3791
:101DE800AD37E82EF9D7AAC0C2F0ABC0C3F0ACC07B
:101DF800C4F0ADC0C5F0B951BA11BB11BC1101E1B5
:101E080096D0FF0EA5250B6EFF0EA6210C6EFF0EB9
:101E1800A7210D6EFF0EA8210E6EC2C00FF0C3C021
:101E280010F0C4C011F0C5C012F00BEC50F00BC09C
:101E3800A9F00CC0AAF00DC0ABF00EC0ACF0FF0EBC
:101E48000001B9250B6EFF0EBA210C6EFF0EBB21E7
:101E58000D6EFF0EBC210E6EC2C00FF0C3C010F095
:101E6800C4C011F0C5C012F00BEC50F00B500001CB
:101E7800A95D0C50AA590D50AB590E50AC5957E3F7
:101E8800FF0EC225A96FFF0EC321AA6FFF0EC42142
:101E9800AB6FFF0EC521AC6FA91DAD6FAA1DAE6F4C
:101EA800AB1DAF6FAC1DB06FFF0EB925B16FFF0E44
:101EB800BA21B26FFF0EBB21B36FFF0EBC21B46F06
:101EC800AD51B115B56FAE51B215B66FAF51B3156F
:101ED800B76FB051B415B86F20EE06F0A351D926EC
:101EE800A451DA22B5C0DEFFB6C0DEFFB7C0DEFF00
:101EF800B8C0DEFF20EE06F0A351D926A451DA229D
:101F0800DE50A55FDE50A65BDE50A75BDD50A85B08
:101F180020EE12F0A351D926A451DA22DECFC6F062
:101F2800DECFC7F0DECFC8F0DECFC9F064D020EE38
:101F38000EF0A351D926A451DA22DECFC6F0DECFA7
:101F4800C7F0DECFC8F0DECFC9F0C651C711C8113F
:101F5800C91143E1A3C0D9FFA4C0DAFFDECF8CF0DA
:101F6800DDCF8DF08E6B8F6B906B916B16EC32F032
:101F78008CC0C6F08DC0C7F08EC0C8F08FC0C9F045
:101F8800C605C711C811C91109E120EE05F0A35112
:101F9800D926A451DA22020EDF6E020CC6290FE1FF
:101FA800C7290DE1C8290BE1C92909E120EE05F08F
:101FB800A351D926A451DA22010EDF6E010C20EEBE
:101FC8000EF0A351D926A451DA22C6C0DEFFC7C03D
:101FD800DEFFC8C0DEFFC9C0DEFF20EE12F0A3514D
:101FE800D926A451DA22C6C0DEFFC7C0DEFFC8C0AA
:101FF800DEFFC9C0DEFFC651C711C811C91101E013
:1020080095D0F1D020EE04F0A351D926A451DA22BC
:10201800DFA228D0A3C0D9FFA4C0DAFFDECF8CF09E
:10202800DDCF8DF0C6C08EF0C7C08FF0C8C090F06D
:10203800C9C091F016EC32F08CC0C6F08DC0C7F064
:102048008EC0C8F08FC0C9F0C651C711C811C911D8
:1020580023E1C2C0A5F0C3C0A6F0C4C0A7F0C5C0A4
:10206800A8F06ED0A3C0D9FFA4C0DAFFDECF44F039
:10207800DDCF45F0C6C046F0C7C047F0C8C048F03D
:10208800C9C049F0C6EC1FF044C0C6F045C0C7F04F
:1020980046C0C8F047C0C9F00001C62907E1C729F2
:1020A80005E1C82903E1C92901E180D7C951C8114F
:1020B800C71104E1020EC65D01E267D7A3C0D9FFCC
:1020C800A4C0DAFF10EE12F0DE50E126DD50E22265
:1020D800E650C65DE650C759E650C859E650C9599A
:1020E80001E353D720EE12F0A351D926A451DA22E6
:1020F800C6C0DEFFC7C0DEFFC8C0DEFFC9C0DEFF46
:1021080020EE06F0A351D926A451DA22C251DE26C8
:10211800C351DE22C451DE22C551DE22C251A55F61
:10212800C351A65BC451A75BC551A85BA551C25D4D
:10213800A651C359A751C459A851C55901E262D73C
:1021480020EE06F0A351D926A451DA22A551DE26A5
:10215800A651DE22A751DE22A851DE22A551A96F81
:10216800010EA615AA6FAB6BAC6BA911AB11AC1124
:102178003AE0A3C0D9FFA4C0DAFFDECF0BF0DDCF71
:102188000CF0C6C00DF0C7C00EF0C8C00FF0C9C033
:1021980010F056EC46F00BC0BEF00CC0BFF00DC0FE
:1021A800C0F00EC0C1F00001BE51BF11C011C11175
:1021B80001E1EBD6A5C0A9F0A6C0AAF0A7C0ABF074
:1021C800A8C0ACF00A0E05D0D890AC33AB33AA3314
:1021D800A933E82EF9D7A951BE27AA51BF23AB517D
:1021E800C023AC51C12320EE06F0A351D926A45137
:1021F800DA22FF0EDE14A96F010EDE14AA6F000E9C
:10220800DE14AB6F000EDE14AC6FA951AA11AB112E
:10221800AC1120E020EE16F0A351D926A451DA2201
:10222800BE51DE1809E1BF51DE1806E1C051DE18C3
:1022380003E1C151DE180EE020EE16F0A351D926B5
:10224800A451DA22BEC0DEFFBFC0DEFFC0C0DEFF81
:10225800C1C0DEFF20EE06F0A351D926A451DA2230
:1022680010EE0AF0A351E126A451E222DE50E65C0A
:10227800DE50E658DE50E658DE50E65801E33DD51C
:1022880020EE06F0A351D926A451DA2210EE0AF066
:10229800A351E126A451E222DECFE6FFDECFE6FF1E
:1022A800DECFE6FFDECFE6FF20EE04F0A351D9260D
:1022B800A451DA22000EDB8A20D564C0A1F065C0E3
:1022C800A2F068C0D9FF69C0DAFFDE6ADD6A62C0C1
:1022D8000CF063C00DF079EC4EF000019C6F9C513E
:1022E80002E09C51120020EE05F06250D92663509E
:1022F800DA22DF5008E020EE05F06250D92663505C
:10230800DA22DF50120020EE04F06250D926635022
:10231800DA22DFA0070C20EE06F06250D9266350BF
:10232800DA22DECF8CF0DECF8DF0DECF8EF0DECF7E
:102338008FF020EE0AF06250D9266350DA22DECF01
:1023480090F0DECF91F0DECF92F0DECF93F08C519B
:10235800905D986F8D519159996F8E5192599A6FDE
:102368008F5193599B6F66508C6F67508D6F8E6B32
:102378008F6B8C51985D8D5199598E519A598F5107
:102388009B5901E34AD298C066F099C067F045D2DC
:1023980020EE06F06250D9266350DA22FF0EDE14D2
:1023A8008C6F010EDE148D6F000EDE148E6F000E22
:1023B800DE148F6F8C518D118E118F1101E0A5D114
:1023C80020EE06F06250D9266350DA22DECF8CF078
:1023D800DECF8DF0DECF8EF0DECF8FF00A0E05D087
:1023E800D8908F338E338D338C33E82EF9D762C073
:1023F800D9FF63C0DAFF10EE02F0DE50E126DD50AF
:10240800E222E750906F90058C15A36FA3516AE103
:1024180020EE06F06250D9266350DA22DE50DE1034
:10242800DE10DE100FE120EE0EF06250D926635068
:10243800DA22DECF9DF0DECF9EF0DECF9FF0DECF3A
:10244800A0F020D062C0D9FF63C0DAFFDECF44F02D
:10245800DDCF45F020EE12F06250D9266350DA2223
:10246800DECF46F0DECF47F0DECF48F0DECF49F0D2
:10247800C6EC1FF044C09DF045C09EF046C09FF0DA
:1024880047C0A0F00001A0519F119E110CE1020E5F
:102498009D5D09E220EE05F06250D9266350DA22EC
:1024A800020EDF6E020C9D290FE19E290DE19F2986
:1024B8000BE1A02909E120EE05F06250D92663500E
:1024C800DA22010EDF6E010C20EE12F06250D926DE
:1024D8006350DA229DC0DEFF9EC0DEFF9FC0DEFF94
:1024E800A0C0DEFF62C0D9FF63C0DAFFDECF0BF009
:1024F800DDCF0CF020EE12F06250D9266350DA22BC
:10250800DECF0DF0DECF0EF0DECF0FF0DECF10F015
:1025180056EC46F00BC0A4F00CC0A5F00DC0A6F018
:102528000EC0A7F00001A451A511A611A71101E141
:10253800B1D7A351A427000EA523A623A72366C0BD
:102548008CF067C08DF0090E8E6FD8908D338C3368
:102558008E2FFBD78CC0A8F08DC0A9F0A851A91167
:1025680001E1C5D0A351A8258C6F000EA9218D6F5C
:1025780062C0D9FF63C0DAFF10EE02F0DE50E12638
:10258800DD50E222E7508E6F8F6B8C518E5D8D513E
:102598008F5912E262C0D9FF63C0DAFF10EE02F071
:1025A800DE50E126DD50E222E7508C6FA3518C5DAE
:1025B800A86FA96BD8A0A907A1C01AF0A2C01BF0E8
:1025C800A4C01CF0A5C01DF0A6C01EF0A7C01FF037
:1025D800A8C020F0A9C021F062C0D9FF63C0DAFF0B
:1025E80010EE01F0DE50E126DD50E222E750B4ECB7
:1025F8004CF0000901E05FD762C0D9FF63C0DAFF81
:1026080010EE04F0DE50E126DD50E222E7505FE0F4
:102618000001A8518C6FA9518D6F8E6B8F6B62C0B2
:10262800D9FF63C0DAFF10EE2AF0DE50E126DD5054
:10263800E222E6CF90F0E6CF91F0E6CF92F0E6CF37
:1026480093F0A451905D946FA5519159956FA6513F
:102658009259966FA7519359976F8C51945D8D51EC
:1026680095598E5196598F51975931E262C0D9FFC9
:1026780063C0DAFF10EE2AF0DE50E126DD50E222D8
:10268800E6CF8CF0E5CF8DF0A4518C5FA5518D5B22
:10269800090ED8908C378D37E82EFBD78C51A125A1
:1026A8000B6E8D51A2210C6E62C0D9FF63C0DAFF98
:1026B800DECF8EF0DDCF8FF02E0E8E250D6E000E44
:1026C8008F210E6E020E106E0F6A59EC54F0A8C0DE
:1026D8008CF0A9C08DF0090ED89000018C378D3789
:1026E800E82EFAD78CC0AAF08DC0ABF079D020EED6
:1026F80016F06250D9266350DA22A4C0DEFFA5C0C6
:10270800DEFFA6C0DEFFA7C0DEFF8C69010E8D6F5D
:1027180020EE06F06250D9266350DA22DECF8EF022
:10272800DDCF8FF08C518E178D518F178E51000889
:10273800AA6F8F51D8A0E82A0208AB6FAA51665C2D
:10274800AB51675804E266C0AAF067C0ABF062C03C
:10275800D9FF63C0DAFFDECF39F0DDCF3AF020EEE3
:1027680016F06250D9266350DA22DECF3BF0DECF76
:102778003CF0DECF3DF0DECF3EF006EC4DF0000938
:1027880001E099D6A1C00BF0A2C00CF000018C6941
:10279800010E8D6F20EE06F06250D9266350DA22C2
:1027A800DECF8EF0DDCF8FF08C518E178D518F17C5
:1027B80062C0D9FF63C0DAFFDECF90F0DDCF91F0C1
:1027C8008E5190278F5191232E0E90250D6E000E5D
:1027D80091210E6EAAC00FF0ABC010F059EC54F066
:1027E800AA51A127AB51A22320EE06F06250D926A8
:1027F8006350DA22AA51DE26AB51DE22000EDE2219
:10280800DE2268C0D9FF69C0DAFFAA51DE26AB51C3
:10281800DD22AA51665EAB51675A6650671001E027
:10282800B7D5000C276E266A15D2275009E100019A
:10283800FE5106E0266A6C6A0A0E92D089907BD215
:10284800020E271807E10001FE5104E0266A6C6AAF
:10285800140E86D01F0E276438D0300E276035D06E
:102868000001FE5132E02750E00F736E266A0F0E0A
:10287800731805E19AC1FDF001019A6BD2D173502A
:10288800200D120EF324D96E020EF420DA6EDE50FB
:10289800DE10DE10DE1003E0030E7364C2D1010EF9
:1028A800FD6F7350140D130EF324D96E010EF4202E
:1028B800DA6E7350140D130EF324E16E010EF4203A
:1028C800E26EE7500409DF6EACD13F0E276414D0E6
:1028D800500E276011D00001FE510EE07350140D08
:1028E800000EF324D96E010EF420DA6E2750C00FC3
:1028F800DF6E266AFD6B95D1310E271807E10001BE
:10290800FE5104E00C0E6C6E1D0E9CD1340E27187F
:1029180007E10001FE5104E06B6A6C6A266A8ED7F3
:10292800350E271808E10001FE5105E0266A0D0E54
:102938006C6EAC0E15D0370E271808E10001FE5159
:1029480005E089800E0E6C6E750E7CD10D0E271871
:1029580009E10001FE5106E0266A020E6C6EBC0E0B
:102968006B6E6CD7100E271807E10001FE5104E0CA
:10297800030E6C6EE90E66D1180E271807E10001E8
:10298800FE5104E0070E6C6E090E5CD13B0E271851
:1029980007E10001FE5104E00E0E6C6E7E0E52D16E
:1029A8003E0E271801E0C7D10001FE5101E1C3D155
:1029B8000F0E6C6E3D0E46D17350140D010EF324AC
:1029C800D96E010EF420DA6E27C0DFFF030E6C6E9D
:1029D800EA0E38D17350140D020EF324D96E010E8D
:1029E800F420DA6E27C0DFFF030E6C6EEB0E2AD1DF
:1029F8007350140D030EF324D96E010EF420DA6E11
:102A080027C0DFFF030E6C6EEC0E1CD17350140D43
:102A1800040EF324D96E010EF420DA6E27C0DFFF0E
:102A2800030E6C6EED0E0ED17350140D050EF324CB
:102A3800D96E010EF420DA6E27C0DFFF030E6C6E2C
:102A4800EE0E00D17350140D060EF324D96E010E4C
:102A5800F420DA6E27C0DFFF7350140D060EF3243E
:102A6800D96E010EF420DA6EDF500B6E0BC00CF03D
:102A78000D6A0E6A0F6A0EC00FF00DC00EF00CC082
:102A88000DF00C6A7350140D050EF324D96E010E67
:102A9800F420DA6EDF50106E10C011F0126A136A5B
:102AA800146A12C014F011C013F0126A116A73503C
:102AB800140D040EF324D96E010EF420DA6EDF50E3
:102AC800156E15C016F0176A186A196A16C019F03B
:102AD800186A176A166A7350140D030EF324D96E18
:102AE800010EF420DA6EDF5016241A6E000E17203D
:102AF8001B6E000E18201C6E000E19201D6E115042
:102B08001A241E6E12501B201F6E13501C20206E9C
:102B180014501D20216E0C501E24226E0D501F20B3
:102B2800236E0E502020246E0F502120256E7350E6
:102B3800140D070EF324D96E010EF420DA6E22C0AC
:102B4800DEFF23C0DEFF24C0DEFF25C0DEFF69D024
:102B58007350140D120EF324D96E010EF420DA6EA0
:102B680027C0DFFF070E6C6E0A0E6CD07350140D71
:102B7800110EF324D96E010EF420DA6E27C0DFFFA0
:102B8800070E6C6E0B0E5ED07350140D100EF324EE
:102B9800D96E010EF420DA6E27C0DFFF070E6C6EC7
:102BA8000C0E50D07350140D0F0EF324D96E010E75
:102BB800F420DA6E27C0DFFF89906B6A6C6ABBD09D
:102BC8006B6A6C6A0001FD6B39D627C000F20F0EE4
:102BD8006C6E3E0E37D027C001F20F0E6C6E3F0EA2
:102BE80031D027C002F20F0E6C6E400E2BD027C0DA
:102BF80003F20F0E6C6E410E25D027C004F20F0EA3
:102C08006C6E420E1FD027C005F20F0E6C6E430E7D
:102C180019D027C006F20F0E6C6E440E13D027C0D1
:102C280007F26B6A6C6A0AD60C0E6C6E1E0E0AD01E
:102C38000C0E6C6E1C0E6B6E0A0E266EFFD50E0EF9
:102C48006C6E760E6B6E77D06B6A6C6A090E266EA8
:102C5800898071D06BC00BF06CC00CF00C5011E087
:102C6800030A13E0040A25E00B0A31E0010A35E003
:102C7800030A39E0010A40E0130A58E03B0A59E028
:102C88005AD00B5001E1D1D556D00B50E90A01E1D9
:102C980093D6030A01E19ED6010A01E1A9D6070AE3
:102CA80001E1B4D6010A01E1BFD6030A01E1CAD69F
:102CB80042D00B50090A01E14BD7030A01E156D76C
:102CC800010A01E161D7070A01E16CD734D00B5042
:102CD8001D0AAAE0030AACE02ED00B50480A01E115
:102CE8006CD7E40A28D00B50750AA9E0030AACE0B7
:102CF800080A01E165D71FD00B503D0A01E165D7ED
:102D0800030A01E168D7010A01E16BD77F0A01E1F3
:102D18006ED7010A01E171D7030A01E174D7010AEC
:102D280001E177D7070A01E17AD705D00B502A0AC3
:102D380002D00B500F0A26501200D251D31101E1D4
:102D4800090CD2C0D9FFD3C0DAFFDE6ADD6A94C1AC
:102D5800C3F195C1C4F11F0ED617C30E666E010EDE
:102D6800676ED40E686ED651FE0B696E09EC00F0E2
:102D78000101C06FC05101E040D2AC0ED76F010E07
:102D8800D86FC30E0001BC6F010EBD6FD4C0BEF07A
:102D9800D5C0BFF075EC41F00101C06FD5C1C1F1DC
:102DA800D6C1C2F1C05105E1C151C21102E1060EFE
:102DB800C06FD6C0D7F01C0E0001D71701E114D19F
:102DC8000101C05113E0040EC01909E1C30E00014E
:102DD800C06F010EC16F52EC4BF00101C06F0001D2
:102DE800D687D5C1C1F1D6C1C2F113D020EE0BF000
:102DF800C151D926C251DA22DF500001D76F110E16
:102E0800D71702E0070E03D0D6A503D0080E01019C
:102E1800C06F0101C05101E002D10001D6A7FFD067
:102E28000101BC6BBD6B210EBE6F460EBF6F20EE5D
:102E38000EF0C151D926C251DA22DF6A20EE0FF016
:102E4800C151D926C251DA22BDC1DFFF20EE10F0F0
:102E5800C151D926C251DA22BEC1DFFF20EE11F0DE
:102E6800C151D926C251DA22BFC1DFFF20EE16F0C8
:102E7800C151D926C251DA22DF6A20EE17F0C151BA
:102E8800D926C251DA22BDC1DFFF20EE18F0C151A8
:102E9800D926C251DA22BEC1DFFF20EE19F0C15196
:102EA800D926C251DA22BFC1DFFF20EE0BF0C15193
:102EB800D926C251DA22DF6A20EE1CF0C151D92688
:102EC800C251DA22DF6A20EE1DF0C151D926C25163
:102ED800DA22DF6A20EE1EF0C151D926C251DA2269
:102EE800DF6A20EE1FF0C151D926C251DA22DF6A0B
:102EF800C3C10BF0C4C10CF0C1C10DF0C2C10EF0CA
:102F08000DEC4CF00BC0B8F10CC0B9F10DC0BAF122
:102F18000EC0BBF1C1C10BF0C2C10CF00D6A0E6A44
:102F28000F6A106A17EC54F0010120EE04F0C35147
:102F3800D926C451DA22010EDF6EB851B911BA117F
:102F4800BB116DE020EE2AF0C351D926C451DA2214
:102F5800DECFBCF1DECFBDF1DECFBEF1DECFBFF1FB
:102F6800C3C18CF0C4C18DF0B8C18EF0B9C18FF067
:102F7800BAC190F0BBC191F0A3EC44F00101C06F5D
:102F8800C0514DE1FF0EB8250001D76FFF0E0101BA
:102F9800B9210001D86FFF0E0101BA210001D96FD4
:102FA800FF0E0101BB210001DA6F010120EE0AF0DA
:102FB800C351D926C451DA22D7C0DEFFD8C0DEFFFC
:102FC800D9C0DEFFDAC0DEFFC3C139F0C4C13AF0B0
:102FD800BCC13BF0BDC13CF0BEC13DF0BFC13EF03D
:102FE80006EC4DF001011AD00101C05118E120EEA4
:102FF8000BF0C151D926C251DA22DFA802D0040E43
:103008000DD00001D6A30BD0010120EE0BF0C15169
:10301800D926C251DA22DFA002D0070EC06F010103
:10302800C05123E10001D6B7D68B010120EE2AF06A
:10303800C351D926C451DA22000110EE1AF0D25138
:10304800E126D351E222DECFE6FFDECFE6FFDECF78
:10305800E6FFDECFE6FF20EE1EF0D251D926D3518F
:10306800DA22C1C1DEFFC2C1DDFF0101C05101E0AA
:10307800C4D0000120EE04F0D251D926D351DA226F
:10308800D6C0DFFF20EE05F0D251D926D351DA227F
:10309800DF6AC3C10BF0C4C10CF0C1C10DF0C2C1DD
:1030A8000EF00DEC4CF0000120EE0EF0D251D926B6
:1030B800D351DA220BC0DEFF0CC0DEFF0DC0DEFFED
:1030C8000EC0DEFF010120EE1DF0C151D926C2510C
:1030D800DA22DF500001D86FD76B010120EE1EF015
:1030E800C151D926C251DA22DF500001D96FD9C0A7
:1030F800DAF0DB6BDC6BDD6BDBC0DDF0DAC0DCF05B
:10310800DB6BDA6B010120EE1FF0C151D926C251E9
:10311800DA22DF500001DE6FDEC0DFF0E06BE16B2A
:10312800E26BDFC0E2F0E16BE06BDF6BDA51DF11DD
:10313800E36FDB51E011E46FDC51E111E56FDD5124
:10314800E211E66FD751E311E76FD851E411E86F48
:10315800000EE511E96F000EE611EA6F010120EE9D
:103168001CF0C151D926C251DA22DF500001E71103
:10317800EB6FE851EC6FE951ED6FEA51EE6F20EE1D
:103188000AF0D251D926D351DA22EBC0DEFFECC0C7
:10319800DEFFEDC0DEFFEEC0DEFF20EE06F0D2510E
:1031A800D926D351DA22DE6ADE6ADE6ADD6A20EECB
:1031B80016F0D251D926D351DA22DE6ADE6ADE6AE7
:1031C800DD6AD2C0D9FFD3C0DAFFC3C1DEFFC4C1F4
:1031D800DDFFD2C0D9FFD3C0DAFF10EE06F0DE5013
:1031E800E126DD50E22220EE02F0D251D926D35159
:1031F800DA22E6CFDEFFE5CFDDFF0101C051120084
:1032080049504810471003E1020E465C10E320EED7
:1032180012F04450D9264550DA22DE50465CDE5082
:103228004758DE504858DE50495801E22FD2020E66
:10323800866F41D246C084F047C085F0D89085316A
:103248004F6E84314E6E4E5084274F50852344C0B4
:1032580039F045C03AF020EE1EF04450D9264550CA
:10326800DA22DECF4EF0DECF4FF0DECF50F0DECFE9
:1032780051F084C052F085C053F0090E546ED890B6
:1032880053325232542EFBD752504E243B6E535079
:103298004F203C6E000E50203D6E000E51203E6EB9
:1032A80006EC4DF00001866F865101E004D24E68AD
:1032B800010E4F6E84C050F085C051F04E5050162C
:1032C8004F50511644C052F045C053F0505052264A
:1032D800515053222E0E5224876F000E5320886FB0
:1032E800844B852B46B004D04AC080F0816B1AD03D
:1032F8004A504E6E4F6A4E3A4F3AF00E4F164E50A5
:103308000F0B4F12F00E4E1687C0D9FF88C0DAFF98
:10331800DF500F0B506E516A4E505010806F4F5057
:103328005110816F87C0D9FF88C0DAFF80C0DFFFE6
:1033380020EE04F04450D9264550DA22010EDF6E03
:1033480044C039F045C03AF020EE1EF04450D9266A
:103358004550DA22DECF4EF0DECF4FF0DECF50F010
:10336800DECF51F084C052F085C053F0090E546E80
:10337800D89053325232542EFBD752504E243B6EC3
:1033880053504F203C6E000E50203D6E000E5120D1
:103398003E6E06EC4DF00001866F865101E08BD140
:1033A8004E68010E4F6E84C050F085C051F04E50EB
:1033B80050164F50511644C052F045C053F050506B
:1033C8005226515053222E0E5224876F000E53203E
:1033D800886F46B00CD04BC04EF00F0E4E1687C00B
:1033E800D9FF88C0DAFFDF50F00B4E1012D04AC068
:1033F8004EF04BC04FF04CC050F04DC051F0050E90
:1034080005D0D890513250324F324E32E82EF9D78B
:103418004E50826F836B87C0D9FF88C0DAFF82C0A5
:10342800DFFF2BD144C039F045C03AF020EE1EF042
:103438004450D9264550DA22DECF4EF0DECF4FF089
:10344800DECF50F0DECF51F04750526E4850536EE9
:103458004950546E556A4E5052243B6E4F5053207B
:103468003C6E505054203D6E515055203E6E06EC37
:103478004DF00001866F865101E01DD14E68010EA6
:103488004F6E46C050F047C051F0D8905036513674
:103498004E5050164F50511644C052F045C053F08C
:1034A80050505226515053222E0E5224876F000E30
:1034B8005320886F87C0D9FF88C0DAFF4AC0DFFF72
:1034C80020EE01F08751D9268851DA224BC0DFFF60
:1034D800D4D044C039F045C03AF020EE1EF0445034
:1034E800D9264550DA22DECF4EF0DECF4FF0DECFC0
:1034F80050F0DECF51F046C052F047C053F048C0FC
:1035080054F049C055F0080E05D0D89055325432C1
:1035180053325232E82EF9D74E5052243B6E4F5058
:1035280053203C6E505054203D6E515055203E6EF5
:1035380006EC4DF00001866F865101E0BCD04E6864
:10354800010E4F6E46C050F047C051F0D89050362B
:103558005136D890503651364E5050164F5051165D
:1035680044C052F045C053F0505052265150532297
:103578002E0E5224876F000E5320886F20EE01F024
:103588008751D9268851DA22DF504F6E4E6A20EED5
:1035980002F08751D9268851DA22DF50506E50C088
:1035A80051F0526A536A546A52C054F051C053F0F1
:1035B800526A516A20EE03F08751D9268851DA22DF
:1035C800DF50556E55C056F0576A586A596A56C04A
:1035D80059F0586A576A566A515056105A6E5250E6
:1035E80057105B6E535058105C6E545059105D6EF6
:1035F8004E505A105E6E4F505B105F6E000E5C109E
:10360800606E000E5D10616E87C0D9FF88C0DAFF5A
:10361800DF505E10626E5F50636E6050646E615082
:10362800656E666A676A686AF00E6514696E665048
:103638004A1267504B1268504C1269504D1287C09D
:10364800D9FF88C0DAFF4AC0DFFF20EE01F08751BA
:10365800D9268851DA224BC0DFFF20EE02F08751CD
:10366800D9268851DA224CC0DFFF20EE03F08751BB
:10367800D9268851DA224DC0DFFF20EE04F04450ED
:10368800D9264550DA22010EDF6E15D044C0D9FF85
:1036980045C0DAFFDF504E6E4F6A4F5001E0C7D584
:1036A8004E50010A01E1C6D5030A01E1BBD6010A61
:1036B80001E10FD7BCD58651120073500C0D500E86
:1036C800F324D96E010EF420DA6E0001CC69CD69BD
:1036D80073500C0D580EF324E16E010EF420E26EC7
:1036E800E6CFCEF0E5CFCFF0CC51CE27CD51CF23CA
:1036F800DE50CE5DCF51800AD06FDE50800AD0599F
:103708004AE373500C0D520EF324D96E010EF420C7
:10371800DA6EDF50CA6FCB6BCC69CD6973500C0D74
:103728005A0EF324D96E010EF420DA6EDF50CE6FF4
:10373800CF6BCC51CE27CD51CF23CA51CE5DCF51BF
:10374800800AD06FCB51800AD05925E373500C0DF5
:10375800530EF324D96E010EF420DA6EDF50CA6FCF
:10376800CB6BCC69CD6973500C0D5B0EF324D96E0D
:10377800010EF420DA6EDF50CE6FCF6BCC51CE271E
:10378800CD51CF23CA51CE5DCF51800AD06FCB51D6
:10379800800AD05961E21F0E0101A66F010EA86FC1
:1037A80089905C0E0001806FFB0E816F73500C0DC9
:1037B800500EF324D96E010EF420DA6EDECF82F0BB
:1037C800DDCF83F073500C0D580EF324D96E010E23
:1037D800F420DA6EDECFCAF0DDCFCBF0FF0ECA25BB
:1037E800846FFF0ECB21856F73500C0D520EF3249E
:1037F800D96E010EF420DA6EDF50866F876B735036
:103808000C0D5A0EF324D96E010EF420DA6EDF5037
:10381800CC6FFF0ECC25886F896BFF0E8923735000
:103828000C0D530EF324D96E010EF420DA6EDF501E
:103838008A6F8B6B73500C0D5B0EF324D96E010EDF
:10384800F420DA6EDF50CD6FFF0ECD258C6F8D6BB7
:10385800FF0E8D23D3EC56F073500C0D530EF3244A
:10386800D96E010EF420DA6EDF500001CA6FCAC0AB
:10387800CBF0CC6BCD6BCE6BCDC0CEF0CCC0CDF049
:10388800CBC0CCF0CB6B73500C0D5B0EF324D96E10
:10389800010EF420DA6EDF50CF6FCFC0D0F0D16BBD
:1038A800D26BD36B73500C0D520EF324D96E010EEC
:1038B800F420DA6EDF50D46FD4C0D5F0D66BD76B56
:1038C800D86BD7C0D8F0D6C0D7F0D5C0D6F0D56B56
:1038D800D551D003F3CFD9F0F4CFDAF0DB6BDC6B42
:1038E800D103F350DA27F450DB23000EDC23D65142
:1038F800D003F350DA27F450DB23000EDC23D55134
:10390800D203F350DB27F450DC23D651D103F35014
:10391800DB27F450DC23D751D003F350DB27F450D6
:10392800DC23D351D503F350DC27D651D203F3500F
:10393800DC27D751D103F350DC27D851D003F350FB
:10394800DC2773500C0D5A0EF324D96E010EF420A7
:10395800DA6EDF50DD6FDDC0DEF0DF6BE06BE16B50
:1039680073500C0D5B0EF324D96E010EF420DA6E41
:10397800DF50E26FE2C0E3F0E46BE56BE66B735097
:103988000C0D500EF324D96E010EF420DA6EDECF42
:10399800E7F0DDCFE8F0E7C0E9F0E8C0EAF0000EB4
:1039A800EABFFF0EEB6FEC6FE951E303F3CFEDF0E5
:1039B800F4CFEEF0EF6BF06BE403F350EE27F45026
:1039C800EF23000EF023EA51E303F350EE27F450FF
:1039D800EF23000EF023E951E503F350EF27F450ED
:1039E800F023EA51E403F350EF27F450F023EB51AE
:1039F800E303F350EF27F450F023E651E903F350C3
:103A0800F027EA51E503F350F027EB51E403F350B4
:103A1800F027EC51E303F350F027EFC0F0F0EEC0CD
:103A2800EFF0EDC0EEF0ED6BED51DE03F3CFF1F00A
:103A3800F4CFF2F0F36BF46BDF03F350F227F4509A
:103A4800F323000EF423EE51DE03F350F227F45073
:103A5800F323000EF423ED51E003F350F327F45061
:103A6800F423EE51DF03F350F327F450F423EF511E
:103A7800DE03F350F327F450F423E151ED03F35040
:103A8800F427EE51E003F350F427EF51DF03F3502E
:103A9800F427F051DE03F350F427D951F125F56FDF
:103AA800DA51F221F66FDB51F321F76FDC51F42183
:103AB800F86FCB51F5250101AD6F0001CC51F6210E
:103AC8000101AE6F0001CD51F7210101AF6F000177
:103AD800CE51F8210101B06F7350200D080EF32468
:103AE8000001A36F020EF420A46FADC1A5F0AEC112
:103AF800A6F0AFC1A7F0B0C1A8F077EC0EF00101B5
:103B0800AC6FAC5112E0660E0001806FFC0E816F45
:103B1800ADC182F0AEC183F0AFC184F0B0C185F011
:103B2800ACC186F0876BD3EC56F073500C0D540E75
:103B3800F324D96E010EF420DA6EADC1DEFFAEC1FA
:103B4800DEFFAFC1DEFFB0C1DEFF0101A86B8990C7
:103B580012005F6E5B5002E0F0EC4AF05E6A5A5069
:103B680001E1B2D15F9E040E5F1803E0140E5F18E6
:103B780007E10101966B976B5B6A070E5A6E070C9B
:103B88003F0E5F1807E1716A0101966B976B5A6ADD
:103B98005B6A12005F0E5F1807E10101A96B966B63
:103BA800976B5A6A5B6A12003F0E5F640BD05F0E18
:103BB8005F6008D0400E5F1805E00101A96B5A6AE2
:103BC8005B6A1200400E5F180AE1010E0101A96F3D
:103BD800716A0101966B976B5A6A5B6A1200200E34
:103BE8005F1801E071D1010E716EF3D7600E5F1896
:103BF80009E10101A95106E0A751080ED8B4030E46
:103C08005E6E7CD0600E5F1809E1715007E001011B
:103C1800A75102E0090E15D0050E13D0680E5F18E3
:103C280009E1715007E01A0E0101976F900E3FD11C
:103C38008980A4D1680E5F1806E10101A95103E04B
:103C4800020E5E6E5BD06A0E5F1807E1715005E0E8
:103C58001A0E0101976FF40E2AD16C0E5F1807E156
:103C6800715005E01A0E0101976F2C0E20D1700ECD
:103C78005F1810E10101A9510DE0A30E0001806F4A
:103C8800FF0E816FD3EC56F0040E5E6E0101966B49
:103C9800976BCED7700E5F1801E070D1715001E1BB
:103CA8006DD11B0E0101976F620E01D18980020E42
:103CB8005F1805E11A0E0101976F920E966F050EB7
:103CC8005F1805E11A0E0101976FAE0E966F070E89
:103CD8005F1805E11A0E0101976FB80E966F080E6E
:103CE8005F1805E11A0E0101976FCC0E966F030E4F
:103CF8005F1802E05F2806E15E6A89900101966B11
:103D0800976B3CD1160E5F1801E038D11A0E0101ED
:103D1800976FA40EBDD0050E5F1805E11A0E0101BC
:103D2800976FF50E966F080E5F1801E027D11A0EEF
:103D38000101976FCC0E966F010EA76F1FD15FC060
:103D480073F01A0E0101976F9B0EA2D05F505D6E43
:103D58005C6A73500C0D500EF324D96E010EF420DA
:103D6800DA6E5CC0DEFF5DC0DDFF1A0E0101976FE1
:103D78009C0E8ED05F505C6E5D6A73500C0D500EB9
:103D8800F324D96E010EF420DA6E5CC0DEFF5DC04C
:103D9800DDFF1A0E0101976F9D0E7AD073500C0D3E
:103DA800520EF324D96E010EF420DA6E5FC0DFFFE5
:103DB8001A0E0101976F9E0E6BD073500C0D530EA7
:103DC800F324D96E010EF420DA6E5FC0DFFF010123
:103DD800966B976B010E62D01A0E0101976FB90EA0
:103DE80066D01A0E0101976FBA0E52D01A0E010151
:103DF800976FBB0E966FCA0E0001806FFE0E816F23
:103E0800D3EC56F00101A86B966B976B48D0010173
:103E1800966B976BCA0E0001806FFE0E816FD3EC14
:103E280056F03DD00101966B976B060E5E6EA6D0DC
:103E38005FC073F00101966B976B5E6A30D0010129
:103E4800A76B1A0E976FF70E966F29D01A0E0101FD
:103E5800976FF70E1DD08990270E0101976F0F0EEF
:103E680017D0180E5F1801E089D01A0E0101976F5C
:103E78002D0E0ED01A0E0101976F2E0E09D01A0EB4
:103E88000101976F2F0E04D01A0E0101976F300EA3
:103E9800966F74D00101966B976B0A0E5E6E8990CF
:103EA8006DD0040E5E6E270E0101976F0F0E966F90
:103EB800BFD68980010104D08990010E0101A76F46
:103EC800966B976B5E6A5AD096C15CF097C15DF0AD
:103ED8005D5007E01A0A09E0010A48E03C0A4CE094
:103EE8004DD05C5001E182D649D05C502C0AB9E033
:103EF800010AC0E0030AC3E0010AC6E01F0ACAE0DB
:103F0800A00A01E1D3D6020A01E119D7090A01E1A1
:103F18001DD7070A01E12ED7010A01E13FD7030A9D
:103F280001E14BD73A0A01E17DD70A0AC5E0160A32
:103F380001E152D7010A01E154D7030A01E156D73A
:103F4800010A01E164D7790A01E17AD60E0A01E192
:103F58006FD7380A01E1DFD6010A01E170D7030AF9
:103F680001E174D7010A01E176D708D05C50580AFC
:103F780098E03A0A9EE002D05C500F0A5EC05AF000
:103F88005B6A120049504810471003E1020E465C74
:103F98000FE320EE12F04450D9264550DA22DE50C5
:103FA800465CDE504758DE504858DE50495808E312
:103FB800010E0001846F000E856B866B876BEFD155
:103FC80000018469856986698769D4D146C088F00B
:103FD80047C089F0D89089314B6E88314A6E4A5073
:103FE80088274B50892344C039F045C03AF020EE69
:103FF8001EF04450D9264550DA22DECF4AF0DECFF3
:104008004BF0DECF4CF0DECF4DF088C04EF089C0CB
:104018004FF0090E506ED8904F324E32502EFBD7CB
:104028004E504A243B6E4F504B203C6E000E4C20A5
:104038003D6E000E4D203E6E06EC4DF0000901E08D
:10404800AED14A68010E4B6E88C04CF089C04DF065
:104058004A504C164B504D1644C04EF045C04FF0D8
:104068004C504E264D504F222E0E4E24D96E000E27
:104078004F20DA6EDF500001826F836B884B892BEB
:1040880044C039F045C03AF020EE1EF04450D9261D
:104098004550DA22DECF4AF0DECF4BF0DECF4CF0CF
:1040A800DECF4DF088C04EF089C04FF0090E506E3B
:1040B800D8904F324E32502EFBD74E504A243B6E8A
:1040C8004F504B203C6E000E4C203D6E000E4D2094
:1040D8003E6E06EC4DF0000901E061D14A68010E20
:1040E8004B6E88C04CF089C04DF04A504C164B506E
:1040F8004D1644C04EF045C04FF04C504E264D5022
:104108004F222E0E4E24D96E000E4F20DA6EDF504D
:10411800516E506A5050000182135150831346B0BB
:1041280006D08251806F0F0E8315816F0FD082C029
:104138004AF083C04BF0040E4C6ED8904B324A3292
:104148004C2EFBD74AC080F04BC081F080C084F071
:1041580081C085F05BD044C039F045C03AF020EE0C
:104168001EF04450D9264550DA22DECF4AF0DECF81
:104178004BF0DECF4CF0DECF4DF047504E6E48503E
:104188004F6E4950506E516A4A504E243B6E4B5008
:104198004F203C6E4C5050203D6E4D5051203E6E8D
:1041A80006EC4DF0000901E0FAD04A68010E4B6EAA
:1041B80046C04CF047C04DF0D8904C364D364A506A
:1041C8004C164B504D1644C04EF045C04FF04C5065
:1041D8004E264D504F222E0E4E2400018A6F000E9F
:1041E8004F208B6F20EE01F08A51D9268B51DA22AD
:1041F800DF504B6E4A6A8AC0D9FF8BC0DAFFDF50A6
:104208004A12000E4AC084F04BC085F0866B876B5B
:10421800C6D044C039F045C03AF020EE1EF04450F4
:10422800D9264550DA22DECF4AF0DECF4BF0DECF7A
:104238004CF0DECF4DF046C04EF047C04FF048C0BE
:1042480050F049C051F0080E05D0D8905132503284
:104258004F324E32E82EF9D74A504E243B6E4B501F
:104268004F203C6E4C5050203D6E4D5051203E6EBC
:1042780006EC4DF0000901E092D04A68010E4B6E41
:1042880046C04CF047C04DF0D8904C364D36D890CB
:104298004C364D364A504C164B504D1644C04EF0D5
:1042A80045C04FF04C504E264D504F222E0E4E24F6
:1042B80000018A6F000E4F208B6F20EE01F08A51AB
:1042C800D9268B51DA22DF504B6E4A6A20EE02F073
:1042D8008A51D9268B51DA22DF504C6E4CC04DF0F2
:1042E8004E6A4F6A506A4EC050F04DC04FF04E6A49
:1042F8004D6A20EE03F08A51D9268B51DA22DF501D
:10430800516E51C052F0536A546A556A52C055F002
:10431800546A536A526A4D505210566E4E5053109A
:10432800576E4F505410586E50505510596E4A5091
:1043380056105A6E4B5057105B6E000E58105C6E3C
:10434800000E59105D6E8AC0D9FF8BC0DAFFDF50AE
:104358005A105E6E5B505F6E5C50606E5D50616EB1
:104368005E50846F5F50856F6050866F0F0E6114CA
:10437800876F15D044C0D9FF45C0DAFFDF504A6EB9
:104388004B6A4B5001E014D64A50010A01E11ED68F
:10439800030A01E1E0D6010A01E13BD709D684C04E
:1043A80044F085C045F086C046F087C047F012004B
:1043B8002A6E1BC041F01CC042F02A5001E0040CD8
:1043C800010E3F6E74B0030CE9D1B1EC56F0000950
:1043D80001E1FDD13F6AFBD1146A156A166A176AB2
:1043E800090EEBEC54F0000901E0F1D12B0E0B6E35
:1043F8000C6A0E6A100E0D6E3FEC52F0000901E1D6
:10440800E6D12B44E846030BE8064DE132C01DF027
:104418003F0E1D161DC01EF01F6A206A216A1FC0AC
:1044280021F01EC020F01F6A1E6A3350236E226AD4
:104438003450246E256A22502426235025222450E5
:104448001E24266E25501F20276E000E2020286E61
:10445800000E2120296E26283B6E000E27203C6E78
:10446800000E28203D6E000E29203E6E3BC01DF038
:104478003CC01EF03DC01FF03EC020F00A0ED89090
:104488001D361E361F362036E82EF9D71BC0D9FF39
:104498001CC0DAFF1DC0DEFF1EC0DEFF1FC0DEFF2E
:1044A80020C0DEFF97D71D6A35AE01D01D2A010E48
:1044B8001D1630C01EF00F0E1E163450030B020DD1
:1044C800F3501E241D24020F406E3150030B1D6E45
:1044D8001E6A0A0ED8901D361E36E82EFBD73250BB
:1044E8001F6E206AD8901F362036D8901F36203687
:1044F8003344E846030B216E226A1F5021262050C0
:1045080022221D5021261E502222212A000E22225C
:1045180021C03BF022C03CF03D6A3E6A40C01DF01D
:10452800F70E1D263BC01EF03CC01FF03DC020F01A
:104538003EC021F01D2A05D0D8901E361F362036E1
:1045480021361D2EF9D734D070A43FD0146A156ACD
:10455800166A176A8D0EEBEC54F0000901E037D1AA
:1045680001EC57F02B0E0B6E0C6A0E6A100E0D6ED6
:104578003FEC52F0000901E12AD1300E406E03D021
:1045880001EC57F040064050FBE135C01DF01D3AE4
:104598000F0E1D16100E1E6E1F6A206A216A1D2A34
:1045A80005D0D8901E361F36203621361D2EF9D755
:1045B8001BC0D9FF1CC0DAFF1EC0DEFF1FC0DEFF14
:1045C80020C0DEFF21C0DEFF05D7146A156A166A0F
:1045D800176A090EEBEC54F0000901E0F8D02B0E35
:1045E8000B6E0C6A0E6A100E0D6E3FEC52F000094D
:1045F80001E1EDD070A232D038C01DF0060E1E6E5B
:10460800D8901D321E2EFCD7FF0E1D2635503F0BAD
:104618001F6E206AD8901F3620363644010B1F269D
:10462800000E20221F2A20221D2A03D0D8901F36D0
:1046380020361D2EFBD71F50216E2050226E236A74
:10464800246A1BC0D9FF1CC0DAFF21C0DEFF22C0CC
:10465800DEFF23C0DEFF24C0DEFFBCD63650030BCE
:104668001D6E1E6AD8901D361E36D8901D361E3611
:10467800D8901D361E363638E842070B1D26000E28
:104688001E221D2A1E223540E8423F0B1F0B1F6EBB
:10469800206A1F2A000E20221D501F02F3CF21F08E
:1046A800F4CF22F02002F35022261E501F02F350AE
:1046B80022262150236E2250246E256A266A1BC0AA
:1046C800D9FF1CC0DAFF23C0DEFF24C0DEFF25C0EF
:1046D800DEFF26C0DEFF7ED641C0D9FF42C0DAFF2A
:1046E80070C0DFFF77D6146A156A166A176A090E52
:1046F800EBEC54F000096BE141C00BF042C00CF048
:104708000E6A100E0D6E3FEC52F0000901E062D601
:104718005ED0146A156A166A176A0A0EEBEC54F032
:10472800000955E141C00BF042C00CF00E6A100EB2
:104738000D6E3FEC52F0E9D7146A156A166A176ACB
:104748003A0EEBEC54F0000942E1040E406E0AD038
:1047580001EC57F041C0D9FF42C0DAFFDF6E414A91
:10476800422A4006405001E135D6F2D7146A156A4C
:10477800166A176A8D0EEBEC54F0000928E101EC7B
:1047880057F041C00BF042C00CF00E6A400E0D6E9F
:104798003FEC52F0BAD7040E3F6E19D01A501D6E76
:1047A8001E6A1E50F8E11D5001E10FD6010A01E111
:1047B80013D6020A01E1C8D6090A8EE0010A93E07D
:1047C800070AA7E0010AB8E0030AD0E0E4D713EC2F
:1047D80057F03F50120055C058F056C059F001012B
:1047E800886B896BF6D154C046F0580E476E57C097
:1047F80048F04750D96EDA6ADECFF6FFDDCFF7FF13
:10480800F86A000EF86E0800F550250AD8A4C3D13E
:104818004750D96EDA6ADE2A000EDD2201018A6B62
:104828008B6B8E6B8F6B8C698D694750D96EDA6A8A
:10483800DECFF6FFDDCFF7FFF86A000EF86E08004E
:10484800F550780AD8B40FD04750D96EDA6ADECF5F
:10485800F6FFDDCFF7FFF86A000EF86E0800F55096
:10486800580AD8A46ED14750D96EDA6ADECFF6FF5F
:10487800DDCFF7FFF86A000EF86E0800F5CF53F0A9
:104888004750D96EDA6ADE2A000EDD224850D96E0A
:10489800DA6ADF50DF2ADF2AD96EDA6ADECF49F01A
:1048A800DDCF4AF049C04BF04AC04CF04D6A4E6A21
:1048B8004F6A506A516A526A46C024F04BC025F0CC
:1048C8004CC026F04DC027F04EC028F04FC029F04C
:1048D80050C02AF051C02BF052C02CF053C02DF01C
:1048E8008DBF01D08E938DBF05D08D5107E18C050A
:1048F800D8B004D0376A010E366E04D08CC136F0B9
:104908008DC137F08AC140F08BC141F08EA904D027
:10491800FE0E4026FF0E412225C038F026C039F091
:1049280027C03AF028C03BF029C03CF02AC03DF02F
:104938002BC03EF02CC03FF0436A1F0E426E0201AE
:10494800A76B6DD04206D8A043060F0E3814446EEC
:10495800456A45BE08D0455004E10A0E445CD8A01B
:1049680002D0570E01D0300E4426000E4522BF0E4D
:104978002E6E2F682D50306E316A2E5030262F50F3
:104988003122315005E11A0E305C02E2010E01D0ED
:10499800000E326E336A32503310D8B425D09F0ED1
:1049A8002E6E2F68200E4410306E000E4510316EAA
:1049B8002E5030262F503122315005E11A0E305C2E
:1049C80002E2010E01D0000E346E356A3450351003
:1049D800D8B40AD044C011F045C012F0D4EC53F05A
:1049E80011C044F012C045F0880E4224D96E020E60
:1049F8004320DA6E44C0DFFF3606D8A037064006EB
:104A0800D8A04106040E2E6ED8903F323E323D3279
:104A18003C323B323A32393238322E2EF5D743BE49
:104A280021D0435004E1020E425CD8A01BD038507C
:104A380039103A103B103C103D103E103F10D8A4DE
:104A480081D737BE05D0375002E13604D8B07AD7BF
:104A580041BE08D0415003E14004D8A003D0010171
:104A68008EB370D701018EA916D04206D8A043068E
:104A7800880E4224D96E020E4320DA6E2DC0DFFF65
:104A88004206D8A04306880E4224D96E020E43205F
:104A9800DA6E300EDF6E24C01AF0880E42241B6EC8
:104AA800020E43201C6E40C01DF041C01EF08EA1B6
:104AB80008D01BC014F01CC015F01AC016F087EC03
:104AC80055F01EBE05D01DC022F01EC023F002D036
:104AD800226A236A206A216A0AD0000E0D6E200E0F
:104AE8000C6E1AC00EF005EC4FF0204A212A225015
:104AF800205C2150800A1F6E2350800A1F58D8A0BE
:104B0800ECD701018EB108D01BC014F01CC015F001
:104B18001AC016F087EC55F01BC00BF01CC00CF047
:104B280038EC54F022500B241A6E23500C201B6EC4
:104B38001AC024F01BC025F024C046F025C047F059
:104B480043D04750D96EDA6ADECFF6FFDDCFF7FFE4
:104B5800F86A000EF86E0800F550250AD8A412D09D
:104B68004750D96EDA6ADE2A000EDD22000E0D6E7D
:104B7800250E0C6E46C00EF005EC4FF0476A010E8C
:104B8800466E22D04750D96EDA6ADE2A000EDD2240
:104B9800466A476A19D04750D96EDA6ADECFF6FFFF
:104BA800DDCFF7FFF86A000EF86E0800F5500C6EBE
:104BB8000D6A46C00EF005EC4FF04750D96EDA6A20
:104BC800DE2A000EDD22DAD7465001018827475039
:104BD800892358C0F6FF59C0F7FF0800F55001E0D7
:104BE80002D688C154F089C155F0120018C0F6FFEA
:104BF80019C0F7FF0800F5CF58F0184A192A58507D
:104C080001E11200250E581804E05850DDEC56F06A
:104C1800EDD7516A526A536A546A18C0F6FF19C030
:104C2800F7FF0800F5CF58F0184A192A300E58181F
:104C38000DE1546A010E536E18C0F6FF19C0F7FF54
:104C48000800F5CF58F0184A192A06D02D0E581822
:104C580003E1546A020EEFD72A0E581843E11A509E
:104C6800D96EDA6A020EDF26DF5CD96EDA6ADECF29
:104C780049F0DECF4AF04AAE0BD049500008496EE1
:104C88004A50D8A0E82A00084A6E546A020E536EA9
:104C980049C051F04AC052F018C0F6FF19C0F7FFDA
:104CA8000800F5CF58F0184A192A22D00A0E5102E6
:104CB800F3CF1BF0F4CF1CF05202F3501C265850CF
:104CC8001B26000E1C22D00E1B24516EFF0E1C202A
:104CD800526E18C0F6FF19C0F7FF0800F5CF58F05C
:104CE800184A192A2F0E586403D0390E5864DED793
:104CF8006C0E581803E04C0E58180AE1538418C07B
:104D0800F6FF19C0F7FF0800F5CF58F0184A192A1E
:104D1800585001E1120058C057F0600E576472D025
:104D2800200E575E6FD01A50D96EDA6A020EDF264F
:104D3800DF5CD96EDA6ADECF41F0DECF42F04F6A2F
:104D4800506A02D04F4A502A4F5041241B6E50508F
:104D580042201C6E1BC0F6FF1CC0F7FF000EF86E49
:104D68000F0EF76403D00800F55005D0F6CFE9FF21
:104D7800F7CFEAFFEF50000904E0E4D7200EDDEC9E
:104D880056F053B20BD04F501B6E50501C6E4F4A0A
:104D9800502A51501B5C52501C58F0E341C00CF093
:104DA80042C00DF0EAEC52F003D0200EDDEC56F0D4
:104DB8004F501B6E50501C6E4F4A502A51501B5C6E
:104DC80052501C5801E312D7F0D71A50D96EDA6A3C
:104DD800DF50DF2ADF2AD96EDA6ADF50DDEC56F0C1
:104DE80005D7446A020E08D0446A080E05D0446A02
:104DF8000A0E02D0446A100E436E19D05850DDECEA
:104E080056F0F4D657501B6E1C6A1C50F7E11B5025
:104E1800420AE7E0010AD9E0070AE9E00B0AE4E000
:104E28001C0A81E0060AE3E00D0AE4E0E7D753A490
:104E380011D01A50D96EDA6A040EDF26DF5CD96EFB
:104E4800DA6ADECF4BF0DECF4CF0DECF4DF0DECFAE
:104E58004EF027D0440E571813E01A50D96EDA6A6C
:104E6800DF50DF2ADF2AD96EDA6ADECF1BF0DDCF0A
:104E78001CF01BC04BF01CC04CF04D6A4E6A11D0A0
:104E88001A50D96EDA6ADF50DF2ADF2AD96EDA6A59
:104E9800DECF4BF0DDCF4CF0000E4CBEFF0E4D6E5A
:104EA8004E6E440E57180CE14EAE0AD04B6C4C1E99
:104EB800D8B04C2A4D1ED8B04D2A000E4E565388F5
:104EC800556A566A4BC045F04CC046F04DC047F095
:104ED8004EC048F045C00BF046C00CF047C00DF07E
:104EE80048C00EF043C00FF044C010F0116A126AB7
:104EF80054EC51F00B50576E45C00BF046C00CF007
:104F080047C00DF048C00EF043C00FF044C010F089
:104F1800116A126A0BEC50F00BC045F00CC046F059
:104F28000DC047F00EC048F0090E57640BD0780E3C
:104F3800581803E03E6A070E02D03E6A270E3D6EFF
:104F48003D50572655501D0FD96EDA6A5750300F0D
:104F5800DF6E554A562A455046104710481005E05E
:104F6800565003E1200E555CB5E353A808D05550C0
:104F78001D0FD96EDA6A2D0EDF6E554A562A55C0B6
:104F88004FF056C050F053B003D0406A200E02D004
:104F9800406A300E3F6E3FC057F003D05750DDECEB
:104FA80056F053B20BD04F501B6E50501C6E4F4AE8
:104FB800502A51501B5C52501C58F0E35506D8A09B
:104FC800560655501D0FD96EDA6ADF50DDEC56F0E3
:104FD8005550561004E0F2D7200EDDEC56F04F5035
:104FE8001B6E50501C6E4F4A502A51501B5C525039
:104FF8001C5801E3FBD5F0D773500C0D530EF32466
:10500800D96E010EF420DA6EDF2A73500C0D530EA0
:10501800F324D96E010EF420DA6EDF500001CA6F56
:10502800CB6BCC69CD6973500C0D5B0EF324D96E34
:10503800010EF420DA6EDF50CE6FCF6BCC51CE2745
:10504800CD51CF23CA51CE5DCF51800AD06FCB51FD
:10505800800AD0594BE273500C0D530EF324D96ECD
:10506800010EF420DA6EDF6A73500C0D520EF32431
:10507800D96E010EF420DA6EDF2A73500C0D520E31
:10508800F324D96E010EF420DA6EDF50CA6FCB6BB1
:10509800CC69CD6973500C0D5A0EF324D96E010EEC
:1050A800F420DA6EDF50CE6FCF6BCC51CE27CD51C6
:1050B800CF23CA51CE5DCF51800AD06FCB51800A21
:1050C800D05914E273500C0D520EF324D96E010E10
:1050D800F420DA6EDF6A73500C0D500EF324D96E8B
:1050E800010EF420DA6EDE2A000EDD2273500C0D5C
:1050F800530EF324D96E010EF420DA6EDF50CA6F16
:10510800CAC0CBF0CC6BCD6BCE6BCDC0CEF0CCC0D3
:10511800CDF0CBC0CCF0CB6B73500C0D5B0EF324F1
:10512800D96E010EF420DA6EDF50CF6FCFC0D0F009
:10513800D16BD26BD36B73500C0D520EF324D96E16
:10514800010EF420DA6EDF50D46FD4C0D5F0D66BE0
:10515800D76BD86BD7C0D8F0D6C0D7F0D5C0D6F0AB
:10516800D56BD551D003F3CFD9F0F4CFDAF0DB6BA0
:10517800DC6BD103F350DA27F450DB23000EDC2379
:10518800D651D003F350DA27F450DB23000EDC238A
:10519800D551D203F350DB27F450DC23D651D10389
:1051A800F350DB27F450DC23D751D003F350DB272F
:1051B800F450DC23D351D503F350DC27D651D20366
:1051C800F350DC27D751D103F350DC27D851D00353
:1051D800F350DC2773500C0D5A0EF324D96E010ED0
:1051E800F420DA6EDF50DD6FDDC0DEF0DF6BE06BE0
:1051F800E16B73500C0D5B0EF324D96E010EF42095
:10520800DA6EDF50E26FE2C0E3F0E46BE56BE66B69
:1052180073500C0D500EF324D96E010EF420DA6E83
:10522800DECFE7F0DDCFE8F0E7C0E9F0E8C0EAF06C
:10523800000EEABFFF0EEB6FEC6FE951E303F3CF0B
:10524800EDF0F4CFEEF0EF6BF06BE403F350EE27E4
:10525800F450EF23000EF023EA51E303F350EE2756
:10526800F450EF23000EF023E951E503F350EF2744
:10527800F450F023EA51E403F350EF27F450F023FD
:10528800EB51E303F350EF27F450F023E651E90321
:10529800F350F027EA51E503F350F027EB51E4030C
:1052A800F350F027EC51E303F350F027EFC0F0F090
:1052B800EEC0EFF0EDC0EEF0ED6BED51DE03F3CF95
:1052C800F1F0F4CFF2F0F36BF46BDF03F350F22755
:1052D800F450F323000EF423EE51DE03F350F227CB
:1052E800F450F323000EF423ED51E003F350F327B9
:1052F800F450F423EE51DF03F350F327F450F42372
:10530800EF51DE03F350F327F450F423E151ED039A
:10531800F350F427EE51E003F350F427EF51DF0385
:10532800F350F427F051DE03F350F427D951F12557
:10533800F56FDA51F221F66FDB51F321F76FDC518B
:10534800F421F86FCB51F525F96FCC51F621FA6F9E
:10535800CD51F721FB6FCE51F821FC6F73500C0D26
:10536800540EF324D96E010EF420DA6EF9C0DEFF74
:10537800FAC0DEFFFBC0DEFFFCC0DEFF7350200D6D
:10538800080EF324A36F020EF420A46F73500C0DC3
:10539800540EF324D96E010EF420DA6EDECFA5F098
:1053A800DECFA6F0DECFA7F0DECFA8F077EC0EF0C8
:1053B8006A6E6A5019E0660E806FFC0E816F73503A
:1053C8000C0D540EF324D96E010EF420DA6EDECFE4
:1053D80082F0DECF83F0DECF84F0DECF85F06AC0C6
:1053E80086F0876BD3EC56F00101A86B120020EE13
:1053F80004F0A351D926A451DA22DECFA7F0DDCFDD
:10540800A8F0A729B06F000EA821B16FB011D8B4C9
:10541800040C20EE0EF0A351D926A451DA22DE5056
:10542800DE10DE10DE1001E1040CB0C0A7F00F0E94
:10543800A71701E094D120EE0EF0A351D926A4516C
:10544800DA22DE2A000EDE22DE22DE2220EE0AF03A
:10545800A351D926A451DA22DE50DE10DE10DE1068
:1054680011E1A3C0D9FFA4C0DAFF10EE08F0DE50A6
:10547800E126DD50E222E650B05DE650B15901E286
:105488006ED1040CB0C0A7F0B1C0A8F0040EA96F8B
:10549800D890A833A733A92FFBD7AA69AB69A3C0B3
:1054A800D9FFA4C0DAFF10EE02F0DE50E126DD508D
:1054B800E222E750AC6FAD6BAA51AC27AB51AD23DC
:1054C800A751AC17A851AD17AC51AD1101E047D1A8
:1054D800A3C0D9FFA4C0DAFFDECF44F0DDCF45F08A
:1054E80020EE0AF0A351D926A451DA22DECF46F0E5
:1054F800DECF47F0DECF48F0DECF49F0C6EC1FF034
:1055080044C0B2F045C0B3F046C0B4F047C0B5F0EF
:105518000001B551B411B31104E1020EB25D01E20C
:10552800020CB22907E1B32905E1B42903E1B52941
:1055380001E1010CA3C0D9FFA4C0DAFF10EE12F0FC
:10554800DE50E126DD50E222E650B25DE650B35966
:10555800E650B459E650B55901E2D2D0A551A6118A
:1055680001E1040CA3C0D9FFA4C0DAFFDECF8CF0A0
:10557800DDCF8DF020EE0AF0A351D926A451DA220E
:10558800DECF8EF0DECF8FF0DECF90F0DECF91F061
:1055980016EC32F08CC0B2F08DC0B3F08EC0B4F00F
:1055A8008FC0B5F0B251B311B411B51101E1070CB8
:1055B800B205B311B411B51101E1020CB22907E12A
:1055C800B32905E1B42903E1B52901E1010CA3C020
:1055D800D9FFA4C0DAFFDECF24F0DDCF25F0D4EC6C
:1055E80042F0000901E0010CA3C0D9FFA4C0DAFF12
:1055F800DECFA7F0DDCFA8F02E0E0001A7250B6E99
:10560800000EA8210C6E0E6A0D6A020E106E0F6A4B
:1056180021EC56F0A3C0D9FFA4C0DAFFDECF0BF00F
:10562800DDCF0CF0B2C00DF0B3C00EF0B4C00FF077
:10563800B5C010F056EC46F0A3C0D9FFA4C0DAFFFD
:1056480010EE2AF0DE50E126DD50E2220BC0E6FF24
:105658000CC0E6FF0DC0E6FF0EC0E6FF0001AE6B12
:10566800AF6B2BD0A3C0D9FFA4C0DAFF10EE04F0B3
:10567800DE50E126DD50E222010EE76EA3C0D9FF1D
:10568800A4C0DAFFDECF24F0DDCF25F0D4EC42F061
:10569800000901E0010CA3C0D9FFA4C0DAFF10EE95
:1056A8002AF0DE50E126DD50E222E62A000EE6224C
:1056B800E622E6220001AE4BAF2BA3C0D9FFA4C05F
:1056C800DAFF10EE02F0DE50E126DD50E222E7506C
:1056D800A76FA86BA751AE5DA851AF59C3E3A3C08C
:1056E800D9FFA4C0DAFF10EE2AF0DE50E126DD5023
:1056F800E222AE51E65EAF51E65A000EE65AE65A8D
:1057080020EE0AF0A351D926A451DA22B2C0DEFF56
:10571800B3C0DEFFB4C0DEFFB5C0DEFFA3C0D9FF53
:10572800A4C0DAFFDECF0BF0DDCF0CF0B2C00DF075
:10573800B3C00EF0B4C00FF0B5C010F056EC46F090
:10574800000120EE0EF0A351D926A451DA220BC095
:10575800DEFF0CC0DEFF0DC0DEFF0EC0DEFF20EE58
:1057680004F0A351D926A451DA22B0C0DEFFB1C09B
:10577800DDFF0F0EB015A76FA86B050ED890A737E1
:10578800A837E82EFBD7A3C0D9FFA4C0DAFFDECF25
:10579800A9F0DDCFAAF0A751A927A851AA232E0E58
:1057A800A927000EAA2320EE12F0A351D926A4514E
:1057B800DA22A9C0DEFFAAC0DDFF000C080E626E67
:1057C800020E636E340E646E0A0E656E020E676E0C
:1057D800666ADD0E686E696A61EC11F00001FF6FA0
:1057E800D10E806FFD0E816FDDC082F0DEC083F0C8
:1057F800D3EC56F00001DF6BE06BDB6BDC6BE16B2D
:10580800E26BE151BD0FD96EDA6ADF6AE151CC0F64
:10581800D96EDA6A000EDF6EE14BE22BE2BFF1D7F8
:10582800E25103E10F0EE15DECE3E36BE46B1ED1A3
:10583800340EE325D96E0A0EE421DA6E0D0EDE1859
:1058480001E0D9D08B0E0B6EFF0E0C6EBD0E0D6EE7
:105858009FEC4DF00B500C1007E1CC0E126E5FEC74
:1058680047F012500101F96F850E0B6EFF0E0C6E9A
:10587800BD0E0D6E9FEC4DF00B500C1007E1CC0ED9
:10588800126E5FEC47F012500101AB6F630E0B6EA6
:10589800FF0E0C6EBD0E0D6E9FEC4DF00B500C10F4
:1058A80007E1CC0E126E5FEC47F012500101A06FB9
:1058B800D10E0B6EFF0E0C6EBD0E0D6E9FEC4DF0F3
:1058C8000B500C1007E1CC0E126E5FEC47F0125033
:1058D8000101AA6F0001E56BE66BAE0E5A6E5B6ABA
:1058E8006A0E5C6EFF0E5D6EE5C05EF0E6C05FF0AE
:1058F800CFEC54F0AE0E0B6E0C6ABD0E0D6E9FEC25
:105908004DF00B500C1018E10F0E0001E503F3CF1A
:10591800ACF0F4CFADF0E603F350AD27340EAC2570
:105928000B6E0C0EAD210C6ECC0E0D6E0E6A106A4D
:105938000F0E0F6E6BEC52F00001E54BE62BE6BF45
:10594800CCD7E65103E1100EE55DC7E3E66B010E27
:10595800E56FAE0E5A6E5B6A710E5C6EFF0E5D6E81
:10596800E5C05EF0E6C05FF0CFEC54F0AE0E0B6E13
:105978000C6ABD0E0D6E9FEC4DF00B500C1018E12B
:105988000F0E0001E503F3CFACF0F4CFADF0E60362
:10599800F350AD27240EAC250B6E0D0EAD210C6E09
:1059A800CC0E0D6E0E6A106A0F0E0F6E6BEC52F075
:1059B8000001E54BE62BE6BFCCD7E65103E1040E28
:1059C800E55DC7E3E16BE26BE151BD0FD96EDA6AC1
:1059D800DF6AE151CC0FD96EDA6A000EDF6EE14B57
:1059E800E22BE2BFF1D7E25103E10F0EE15DECE3F8
:1059F800DB6BDC6B15D0340EE325D96E0A0EE4217F
:105A0800DA6E0A0EDE1830E0340EE325D96E0A0E7F
:105A1800E421DA6E200EDE1806E1DC6B010EDB6F86
:105A2800DF6BE06B21D0DB51DC1109E0340EE3259C
:105A3800D96E0A0EE421DA6EDF51CC0F08D0340E8D
:105A4800E325D96E0A0EE421DA6EDF51BD0FE16E4F
:105A5800E26ADFCFE7FFE0BF05D0E05105E10F0EB6
:105A6800DF5D02E2DF4BE02BE34BE42BDD51E35D2E
:105A7800DE51E45901E2DCD6C10E806FFD0E816F64
:105A8800A0C182F0836BD3EC56F02E0E0001806F1C
:105A9800FE0E816FF9C182F0836BD3EC56F01F0EB6
:105AA8000001806FFE0E816FABC182F0836BD3EC77
:105AB80056F00001E56BE66B4D0E806FFD0E816FB1
:105AC800E5C082F0E6C083F00F0EE503F3CFACF03B
:105AD800F4CFADF0E603F350AD27340EAC25846F58
:105AE8000C0EAD21856FD3EC56F00001E54BE62B8B
:105AF800E6BFE2D7E65103E1100EE55DDDE3E46BB6
:105B0800010EE36F5E0E806FFD0E816FE3C082F0C1
:105B1800E4C083F00F0EE303F3CFACF0F4CFADF0A5
:105B2800E403F350AD27240EAC25846F0D0EAD2190
:105B3800856FD3EC56F00001E34BE42BE4BFE2D7CA
:105B4800E45103E1040EE35DDDE3590E806FFB0EC3
:105B5800816FD3EF56F043C024F044C025F0D4EC55
:105B680042F04D6E4D5001E08ED143C0D9FF44C084
:105B7800DAFF030EDE1801E076D120EE05F043507F
:105B8800D9264450DA22DE0401E06DD12E0E4324DA
:105B98000B6E000E44200C6E0E6A0D6A020E106E1B
:105BA8000F6A21EC56F022EE2CF04350D9264450CF
:105BB800DA22550EDF6E22EE2DF04350D9264450DE
:105BC800DA22AA0EDF6E20EE2EF04350D92644507A
:105BD800DA22520EDF6E20EE2FF04350D9264450C1
:105BE800DA22520EDF6E20EE30F04350D9264450B0
:105BF800DA22610EDF6E20EE31F04350D926445090
:105C0800DA22410EDF6E22EE12F04350D9264450BC
:105C1800DA22720EDF6E22EE13F04350D92644507A
:105C2800DA22720EDF6E22EE14F04350D926445069
:105C3800DA22410EDF6E22EE15F04350D926445089
:105C4800DA22610EDF6E20EE0EF04350D926445062
:105C5800DA2212EE16F04350E1264450E222DFCF5A
:105C6800E7FF22EE17F04350D9264450DA2210EE0F
:105C78000EF04350E1264450E222E6CF45F0E5CF4E
:105C880046F046C045F0466A4550DF6E22EE18F0F1
:105C98004350D9264450DA2210EE0EF04350E12644
:105CA8004450E222E6CF45F0E6CF46F0E6CF47F093
:105CB800E6CF48F0110E05D0D89048324732463228
:105CC8004532E82EF9D74550DF6E22EE19F04350E1
:105CD800D9264450DA2210EE0EF04350E126445003
:105CE800E222E6CF45F0E6CF46F0E6CF47F0E6CF32
:105CF80048F0190E05D0D89048324732463245321E
:105D0800E82EF9D74550DF6E20EE0AF04350D92629
:105D18004450DA2212EE1AF04350E1264450E222AF
:105D2800DFCFE7FF22EE1BF04350D9264450DA229A
:105D380010EE0AF04350E1264450E222E6CF45F047
:105D4800E5CF46F046C045F0466A4550DF6E22EE84
:105D58001CF04350D9264450DA2210EE0AF0435082
:105D6800E1264450E222E6CF45F0E6CF46F0E6CF02
:105D780047F0E6CF48F0110E05D0D89048324732A8
:105D880046324532E82EF9D74550DF6E22EE1DF037
:105D98004350D9264450DA2210EE0AF04350E12647
:105DA8004450E222E6CF45F0E6CF46F0E6CF47F092
:105DB800E6CF48F0190E05D0D8904832473246321F
:105DC8004532E82EF9D74550DF6E20EE1AF04350E1
:105DD800D9264450DA22DECF45F0DECF46F0DECFBA
:105DE80047F0DECF48F04528496E000E46204A6E3F
:105DF800000E47204B6E000E48204C6E20EE2AF015
:105E08004350D9264450DA2249C0DEFF4AC0DEFF9B
:105E18004BC0DEFF4CC0DEFF2E0E43241A6E000E70
:105E280044201B6E20EE2AF04350D9264450DA2233
:105E3800DECF1CF0DECF1DF0DECF1EF0DECF1FF070
:105E4800216A010E206E20EE01F04350D9264450FD
:105E5800DA22DF50DAEC48F020EE05F04350D9267C
:105E68004450DA22DF6A1A6A1B6A1C6A20EE01F0C3
:105E78004350D9264450DA22DF50DCEC21F00009E7
:105E880002E0010E4D6E4D5012008980F6EC3FF095
:105E9800CAC0B1F1CBC0B2F10101B151B2111AE0DF
:105EA8007350140D130EF324D96E010EF420DA6E1C
:105EB8007350140D130EF324E16E010EF420E26EFC
:105EC800E7500409DF6EB4EC55F0B1C1E1F0B2C19E
:105ED800E2F01200AA515CE073505AE17350140DBD
:105EE800070EF324D96E010EF420DA6E84C1E8F0AF
:105EF80085C1E9F086C1EAF00001E76B000EE725ED
:105F0800EB6F010EE821EC6F000EE921ED6F000E3A
:105F1800EA21EE6FDE50EB193BE1DE50EC1938E177
:105F2800DE50ED1935E1DE50EE1932E1EDEC50F0BE
:105F38000FC0B5F110C0B6F111C0B7F112C0B8F179
:105F4800000EE8CF34FA2AEE35F0B8C1DFFFE8CF0B
:105F580036FA2AEE37F0B7C1DFFFE8CF38FA2AEE73
:105F680039F0B6C1DFFFE8CF3AFA2AEE3BF0B5C107
:105F7800DFFF0101F793010E5B6E5A6A3DEC3DF0BD
:105F8800F7930001FD6B8990FDC0E1F0E26B120010
:105F98007350140D0F0EF324D96E010EF420DA6E2F
:105FA800DECFE3F0DECFE4F0DECFE5F0DECFE6F0E3
:105FB800E4C0E3F0E5C0E4F0E6C0E5F00001E66B1C
:105FC800E3C0ACF1E4C0ADF17350140D0F0EF3242F
:105FD800D96E010EF420DA6EDECFE3F0DDCFE4F007
:105FE800E3510101B36FB46BF793AE6BAF6B61D044
:105FF800E369E469ACC1E5F0ADC1E6F0E351E5273A
:10600800E451E6230101AE510001E5190AE101015D
:10601800AF510001E61905E10101B351B41101E1E5
:10602800F7837350200D080EF324626E020EF420DD
:10603800636E340E646E0A0E656E010E676E666AD4
:10604800B90E686E010E696E61EC11F00101B06F56
:10605800B05101E025D7B9C15AF0BAC15BF03DECA7
:106068003DF07350140D070EF324D96E010EF42081
:10607800DA6E000EDE240001E36F010EDE20E46F0D
:10608800000EDE20E56F000EDE20E66F7350140D63
:10609800070EF324D96E010EF420DA6EE3C0DEFF9A
:1060A800E4C0DEFFE5C0DEFFE6C0DEFF0101AE4B67
:1060B800AF2BAC51AE5DAF51800A0001E36F010117
:1060C800AD51800A0001E35993E30101B4BF4FD0F9
:1060D800B45102E1B3054BE37350200D080EF324CD
:1060E800626E020EF420636E340E646E0A0E656EE4
:1060F800B3C166F0B4C167F0B90E686E010E696E7F
:1061080061EC11F00101B06FB05101E0C9D6B9518D
:10611800BA1101E1C5D6F783B3C15AF0B4C15BF037
:106128003DEC3DF07350140D070EF324D96E010EAB
:10613800F420DA6E000EDE240001E36F010EDE208B
:10614800E46F000EDE20E56F000EDE20E66F735070
:10615800140D070EF324D96E010EF420DA6EE3C095
:10616800DEFFE4C0DEFFE5C0DEFFE6C0DEFF0101C2
:1061780007D71550D96EDA6ADECF22F0DDCF23F0CB
:1061880002D0224A232A22C0F6FF23C0F7FF000EBE
:10619800F86E0F0EF76403D00800F55005D0F6CF5F
:1061A800E9FFF7CFEAFFEF502F0AEBE022C0F6FF36
:1061B80023C0F7FF000EF86E0F0EF76403D0080037
:1061C800F55005D0F6CFE9FFF7CFEAFFEF505C0AAC
:1061D800D8E020EE14F01350D9261450DA22DECF7E
:1061E80024F0DDCF25F024C00BF025C00CF00E6A9A
:1061F800200E0D6E106A0B0E0F6E21EC56F01E6A03
:106208001EC026F0276A26C01CF027C01DF0206A91
:10621800080E1F6E1C502224166E1D502320176E68
:1062280016C0F6FF17C0F7FF000EF86E0F0EF764E2
:1062380003D00800F55005D0F6CFE9FFF7CFEAFF05
:10624800EF50286E1C4A1D2A200E2864A7D02F0E56
:10625800281801E1A3D05C0E281801E19FD02E0E6A
:10626800281805E01F50265C2050275814E3080E14
:106278001F182010D8A4060C2E0E281801E0060CB2
:10628800276A080E266E206A0B0E1F6ED8901E36DF
:10629800D8901E36BFD77F0E286402D0030E1E1278
:1062A800800E286403D09F0E286406D0DF0E286471
:1062B8004CD0FD0E286049D01C502224166E1D506B
:1062C8002320176E16C0F6FF17C0F7FF000EF86EF2
:1062D8000F0EF76403D00800F55005D0F6CFE9FF9C
:1062E800F7CFEAFFEF50216E1C4A1D2A3F0E2164AA
:1062F80003D07E0E216406D07F0E2164060CFD0EAD
:106308002160060C166817681FC018F020C019F025
:1063180016501826175019221850265C195027585D
:1063280001E3060C26502424D96E27502520DA6E66
:1063380028C0DFFF264A272A26502424D96E275052
:106348002520DA6E21C0DFFF26D06A0E0B6EFE0E06
:106358000C6E28C00DF00E6AB3EC54F00B500C1004
:1063680001E0060C400E286405D05B0E286002D0C0
:106378001E8209D0600E286406D07B0E286003D0E8
:106388001E80200E285E26502424D96E27502520F2
:10639800DA6E28C0DFFF264A272A3CD71C50222461
:1063A800166E1D502320176E1550D96EDA6A16C066
:1063B800DEFF17C0DDFF200E286403D01A6A1B6AAF
:1063C80003D01B6A040E1A6E1AC028F02650271034
:1063D80001E1060C24C0D9FF25C0DAFFE50EDE185E
:1063E80006E124C0D9FF25C0DAFF050EDF6E080ECE
:1063F8001F18201004E1D8901E36D8901E361E5063
:10640800030BE80601E128881E500C0B040A01E181
:10641800288620EE0BF02450D9262550DA2228C0F1
:10642800DFFF000C8E518F119011911128E120EEA1
:106438000AF08C51D9268D51DA22DECF97F0DECFC3
:1064480098F0DECF99F0DECF9AF097519811991114
:106458009A110FE020EE12F08C51D9268D51DA22D4
:10646800DE50975DDE509859DE509959DE509A59A2
:1064780052E3010E976F986B996B9A6B4CD08CC056
:1064880044F08DC045F08EC046F08FC047F090C0F4
:1064980048F091C049F0C6EC1FF044C09FF045C0D9
:1064A800A0F046C0A1F047C0A2F00001A251A1117E
:1064B800A01109E1020E9F5D06E2010E8C6F8D6B43
:1064C8008E6B8F6B000C9F290FE1A0290DE1A1298C
:1064D8000BE1A22909E19FC08CF0A0C08DF0A1C0FA
:1064E8008EF0A2C08FF0120020EE12F08C51D92647
:1064F8008D51DA22DE509F5DDE50A059DE50A15941
:10650800DE50A259E8E38EC097F08FC098F090C093
:1065180099F091C09AF097C09BF098C09CF099C0F0
:106528009DF09AC09EF09B2B000E9C239D239E23DA
:1065380020EE12F08C51D9268D51DA22DE509B5D67
:10654800DE509C59DE509D59DE509E5911E3020ED3
:106558009B6F9C6B9D6B9E6B9A519911981108E1EA
:10656800020E975D05E28C6B8D6B8E6B8F6B120044
:106578008CC044F08DC045F09BC046F09CC047F0ED
:106588009DC048F09EC049F0C6EC1FF044C09FF083
:1065980045C0A0F046C0A1F047C0A2F000019F513D
:1065A800A011A111A2111AE09F2906E1A02904E176
:1065B800A12902E1A2298FE09F05A011A111A21132
:1065C8008AE097519B19AFE198519C19ACE1995118
:1065D8009D19A9E19A519E19C6E0A5D78CC044F02F
:1065E8008DC045F09BC046F09CC047F09DC048F068
:1065F8009EC049F04A684B684C680F0E4D6E04EC1B
:1066080019F0966F96511CE18E518F1190119111CE
:1066180017E08CC044F08DC045F08EC046F08FC0A6
:1066280047F090C048F091C049F09BC04AF09CC028
:106638004BF09DC04CF09EC04DF004EC19F0966FE5
:10664800965130E120EE0AF08C51D9268D51DA228C
:106658009BC0DEFF9CC0DEFF9DC0DEFF9EC0DEFF4C
:1066680020EE0EF08C51D9268D51DA22DE2806E173
:10667800DE2804E1DE2802E1DE2821E020EE0EF02B
:106688008C51D9268D51DA22DE06000EDE5ADE5AEA
:10669800DE5A20EE05F08C51D9268D51DA22000EF3
:1066A800DB800DD0960507E0010E9B6F000E9C6BFA
:1066B8009D6B9E6B04D09B699C699D699E699BC07C
:1066C8008CF09CC08DF09DC08EF09EC08FF01200A3
:1066D80020EE04F06250D9266350DA2264C0DEFF4F
:1066E80065C0DDFF20EE06F06250D9266350DA223D
:1066F800DECF99F0DECF9AF0DECF9BF0DECF9CF0B4
:10670800000199059A119B119C11D8B4020C62C022
:10671800D9FF63C0DAFF10EE12F0DE50E126DD503B
:10672800E222E650995DE6509A59E6509B59E650A8
:106738009C5901E3020C99519A119B119C1121E17A
:1067480062C0D9FF63C0DAFFDECF8CF0DDCF8DF0F9
:106758008CC0D9FF8DC0DAFF030EDE1812E162C0CB
:10676800D9FF63C0DAFF10EE22F0DE50E126DD50DB
:10677800E222E6CF99F0E6CF9AF0E6CF9BF0E6CF9B
:106788009CF099519A119B119C1123E162C0D9FF89
:1067980063C0DAFF10EE08F0DE50E126DD50E22299
:1067A800E650645CE650655801E3020C62C0D9FF0C
:1067B80063C0DAFF10EE22F0DE50E126DD50E2225F
:1067C800E6CF95F0E6CF96F0E6CF97F0E6CF98F0D3
:1067D80074D062C0D9FF63C0DAFF10EE02F0DE5059
:1067E800E126DD50E222E750100DF3CF93F0F4CF0D
:1067F80094F044D062C0D9FF63C0DAFFDECF44F022
:10680800DDCF45F099C046F09AC047F09BC048F0EC
:106818009CC049F0C6EC1FF044C099F045C09AF0FE
:1068280046C09BF047C09CF00001992907E19A29CE
:1068380005E19B2903E19C2901E1010C9C519B1175
:106848009A1104E1020E995DD8A0020C62C0D9FF2A
:1068580063C0DAFF10EE12F0DE50E126DD50E222CE
:10686800E650995DE6509A59E6509B59E6509C5976
:1068780001E3020C9351645E9451655A9351645C30
:1068880094516558B7E262C0D9FF63C0DAFFDECF22
:106898000BF0DDCF0CF099C00DF09AC00EF09BC044
:1068A8000FF09CC010F056EC46F00BC095F00CC0F1
:1068B80096F00DC097F00EC098F020EE0AF06250E6
:1068C800D9266350DA2299C0DEFF9AC0DEFF9BC04A
:1068D800DEFF9CC0DEFF00019551961197119811BB
:1068E80001E1020C64C08CF065C08DF0040E8E6F5F
:1068F800D8908D338C338E2FFBD78C5195258F6F85
:106908008D519621906F000E9721916F000E98215E
:10691800926F20EE0EF06250D9266350DA228FC0B3
:10692800DEFF90C0DEFF91C0DEFF92C0DEFF0F0EDB
:1069380064148C6F8D6B050ED8908C378D37E82ECC
:10694800FBD762C0D9FF63C0DAFFDECF8EF0DDCFA0
:106958008FF08C518E278D518F232E0E8E27000E8F
:106968008F2320EE12F06250D9266350DA228EC0AF
:10697800DEFF8FC0DDFF000C000E0001F66F0A0E6F
:10698800F56F000EF46F050EF36F2AD1F66B140E37
:10699800F56F1ED1EE0E0C6EFC0E0D6EEAEC52F089
:1069A80082B204D00001F66B1E0EF56F150E0001C1
:1069B800F26F4B0EF16FBE0EE82EFED7F12FFCD70B
:1069C800F22FFAD700F004D1E40E0C6EFE0E0D6E15
:1069D800EAEC52F0060E0001D26F080ED36F5B0E80
:1069E800D46FFB0ED56FD66B54EC4DF0FF6FFF5193
:1069F8003DEC53F00001FF51D9E1F66B230ED5D7DA
:106A08003D0E0C6EFE0E0D6EEAEC52F0080E000103
:106A1800D26F020ED36F070ED46FFF0ED56F010E23
:106A2800D66FA1EC16F00001FF6FFF513DEC53F05B
:106A38000001FF510AE1E2EC2BF0080E5B6E020E3A
:106A48005C6E3DEC55F00001FF6FFF513DEC53F0DB
:106A5800000E0001F66F280EF56F0101A0510CE140
:106A6800F86B340E5A6E0C0E5B6EB00E5C6EFE0E3A
:106A78005D6ECFEC54F00DD0E30E0001806FFB0E7D
:106A8800816FA0C182F0836BF8C184F0856BD3EC71
:106A980056F04C0E0001806FFE0E816F0101F85117
:106AA8000F0D340EF3240001826F0C0EF420836F57
:106AB800D3EC56F07BD77E0E806FFC0E816F010100
:106AC800F8510F0D340EF3240001826F0C0EF420E0
:106AD800836FD3EC56F0080E0001D26F020ED36F0D
:106AE8000101F8510F0D340EF3240001D46F0C0E80
:106AF800F420D56F030ED66FA1EC16F00001FF6FDE
:106B0800FF5103E1F66B3C0EF56F040EFF1901E02F
:106B18004DD7F66B320E49D73B0E806FFD0E816F55
:106B28000101F8510F0D340EF3240001826F0C0E91
:106B3800F420836FD3EC56F0080E0001D26F020EDA
:106B4800D36F0101F8510F0D340EF3240001D46FF7
:106B58000C0EF420D56F070ED66FA1EC16F00001CD
:106B6800FF6FFF5101E022D7F66B3C0E1ED7020ED5
:106B7800806FFD0E816F0101F8510F0D340EF32463
:106B88000001826F0C0EF420836FD3EC56F00001E5
:106B9800F06B010EEF6F010CF5C0F1F0F6C0F2F0EA
:106BA800F25116E1F1510A0A01E1F0D61E0A01E19B
:106BB800F1D60A0A01E108D73D0A01E121D70B0AFB
:106BC80001E179D7050A04E01F0AA6E00E0ACFE022
:106BD800140E0001F519F61103E0F307D8A0F40725
:106BE800F4BF04D0F451D8E1F305D6E2EF6BF06BB3
:106BF8001200340E0101B86F0A0EB96FEAC00BF02B
:106C0800EBC00CF038EC54F00B500101AC6FCA0E1D
:106C18000001A36FA46BA56BA66BA76BA86B77ECA1
:106C28000EF00101B56FB5510DE0350E0001806F12
:106C3800FC0E816FD3EC56F00001CA6BCB6BCC6BAA
:106C4800CD6B1200CA0E626E636AB8C164F0B9C136
:106C580065F0010E676E666AB30E686E010E696EA6
:106C680061EC11F00101B56FB55108E0C30E0001E8
:106C7800806FFC0E816FD3EC56F0DED7B8C1D9FF18
:106C8800B9C1DAFF800EDE1808E06F0E0001806FD0
:106C9800FD0E816FD3EC56F0CFD720EE0AF0B85135
:106CA800D926B951DA22DF500001ED6FEC6B0101F2
:106CB80020EE0BF0B851D926B951DA22DF50000185
:106CC800EC250101B16F000E0001ED210101B26F49
:106CD800AC0E0001806FFC0E816FB1C182F0B2C1B1
:106CE80083F0D3EC56F0CA0E0001A36FA46B010128
:106CF800B1510001ED6FEC6BECC0A5F0EDC0A6F052
:106D0800A76BA86B77EC0EF00101B56FB55194E154
:106D1800CA0E626E636AB8C164F0B9C165F0010E4B
:106D2800676E666AB30E686E010E696E61EC11F0EB
:106D38000101B56FB55180E1B66BB76BEAC00BF0D6
:106D4800EBC00CF0B6C1ECF0B7C1EDF0050ED89071
:106D58000001EC37ED37E82EFAD7EC510101B825E0
:106D68000D6E0001ED510101B9210E6EACC10FF09D
:106D7800106A32EC4EF00B500C105DE1B6C1ECF02D
:106D8800B7C1EDF0050ED8900001EC37ED37E82ECD
:106D9800FAD7B8C1EEF0B9C1EFF0EC51EE27ED51DA
:106DA800EF230E0EEE25D96E000EEF21DA6EDF50BE
:106DB800F16FF06BB6C1F2F0B7C1F3F0050ED890E1
:106DC800F237F337E82EFBD7B8C1F4F0B9C1F5F0C4
:106DD800F251F427F351F5230F0EF425D96E000E66
:106DE800F521DA6EDF50F66FF76BF051F627F151A7
:106DF800F723F6C0ADF1F7C0AEF10101000EAEBF4A
:106E0800FF0EAF6FB06F5B0E0001806FFE0E816FDB
:106E1800ADC182F0AEC183F0AFC184F0B0C185F0DE
:106E2800D3EC56F0ADC1CAF0AEC1CBF0AFC1CCF0D7
:106E3800B0C1CDF01200B64BB72BB7BF7FD7B75153
:106E480005E10F0EB65D01E3F7D678D7F5D6000158
:106E5800BB6B010EBA6F8980BC6BBD6BBE6BBF6B21
:106E6800FED07350200D080EF324626E020EF4203B
:106E7800636E340E646E0A0E656E010E676E666A86
:106E8800C60E686E696A61EC11F00001C86FC851DE
:106E980018E0180E0101A66F010EA86F0001C76B5C
:106EA800C66F810E806FFB0E816F73C082F0836B9B
:106EB800C8C084F0856BC6C086F0C7C087F0D3EC25
:106EC80056F00101AA514BE073500C0D540EF324F7
:106ED800D96E010EF420DA6E84C1B1F085C1B2F02A
:106EE80086C1B3F00001B06B000EB025B46F010E7F
:106EF800B121B56F000EB221B66F000EB321B76F86
:106F0800DE50B4192CE1DE50B51929E1DE50B6196E
:106F180026E1DE50B71923E1EDEC50F00FC0C2F0C6
:106F280010C0C3F011C0C4F012C0C5F0000EE8CF05
:106F380034FA2AEE35F0C5C0DFFFE8CF36FA2AEE7C
:106F480037F0C4C0DFFFE8CF38FA2AEE39F0C3C003
:106F5800DFFFE8CF3AFA2AEE3BF0C2C0DFFF0101BB
:106F6800F793A65101E0F783C6C05AF0C7C05BF09B
:106F78003DEC3DF05AC0C0F05BC0C1F00001C0510B
:106F8800BC27C151BD23000EBE23BF2381AC6CD0EA
:106F9800C651C01903E1C751C11925E0BA6BBB6BD3
:106FA80073500C0D530EF324D96E010EF420DA6ED3
:106FB800DF500EE173500C0D500EF324D96E010E04
:106FC800F420DA6EDE50DE1003E1050EF9EC56F01F
:106FD800D70E0001806FFE0E816FC0C082F0C1C065
:106FE80083F0D3EC56F07CEC56F00EEC57F00B50D7
:106FF8000C1004E0010E0101A86F36D00001B96B36
:10700800050EB86F1CD0680E0001AC6FE40EE82EB8
:10701800FED7AC2FFCD700F00EEC57F00B500C103D
:107028000EE00001BA6BBB6BE10E806FFD0E816F45
:10703800B8C082F0B9C083F0D3EC56F008D0000194
:10704800B807D8A0B907B829DEE1B929DCE10EEC08
:1070580057F00B500C1003E00001BA6BBB6B00013A
:10706800BA51BB1101E0FDD60101A86B899012004D
:1070780020EE04F04450D9264550DA22DF6A20EE8B
:107088002AF04450D9264550DA22DE68DE68DE68E8
:10709800DD6844C039F045C03AF046C03BF047C00F
:1070A8003CF048C03DF049C03EF006EC4DF0000908
:1070B80001E0030C22EE2DF04450D9264550DA2287
:1070C800DF504B6E4A6A22EE2CF04450D9264550C8
:1070D800DA22DF504A12550E4A1803E1AA0E4B185D
:1070E80001E0020C20EE65F04450D9264550DA2222
:1070F800DF504B6E4A6A20EE66F04450D926455060
:10710800DA22DF504C6E4CC04DF04E6A4F6A506A1E
:107118004EC050F04DC04FF04E6A4D6A20EE67F0F9
:107128004450D9264550DA22DF50516E51C052F0F2
:10713800536A546A556A52C055F0546A536A526A7F
:107148004D505210566E4E505310576E4F505410AB
:10715800586E50505510596E4A5056105A6E4B5032
:1071680057105B6E000E58105C6E000E59105D6E65
:1071780020EE64F04450D9264550DA22DF505A10E8
:107188005E6E5B505F6E5C50606E5D50616E5E500F
:10719800626E5F50636E6050646E656A460E621878
:1071A80008E1410E631805E1540E6418651001E109
:1071B800000C20EE81F04450D9264550DA22DF50E9
:1071C8004B6E4A6A20EE82F04450D9264550DA22A6
:1071D800DF504C6E4CC04DF04E6A4F6A506A4EC03C
:1071E80050F04DC04FF04E6A4D6A20EE83F0445087
:1071F800D9264550DA22DF50516E51C052F0536AF9
:10720800546A556A52C055F0546A536A526A4D50CE
:107218005210566E4E505310576E4F505410586EB1
:1072280050505510596E4A5056105A6E4B505710C0
:107238005B6E000E58105C6E000E59105D6E20EEED
:1072480080F04450D9264550DA22DF505A105E6E3D
:107258005B505F6E5C50606E5D50616E5E50626E3A
:107268005F50636E6050646E656A460E621808E18E
:10727800410E631805E1540E6418651001E1000C15
:10728800010C4EC00CF04FC00DF079EC4EF0546E6E
:10729800545001E0FDD020EE04F04E50D9264F5056
:1072A800DA22DFAAF5D04EC0D9FF4FC0DAFFDECF11
:1072B80039F0DDCF3AF020EE1AF04E50D9264F5073
:1072C800DA22DECF3BF0DECF3CF0DECF3DF0DECF82
:1072D8003EF006EC4DF0546E545001E0D9D020EE4B
:1072E8001EF04E50D9264F50DA22DECF59F0DDCFAE
:1072F8005AF020EE0BF05950D9265A50DA22000ED7
:10730800DB8A20EE0AF04E50D9264F50DA2210EED2
:107318001CF05950E1265A50E222DFCFE7FF20EE59
:107328001DF05950D9265A50DA2210EE0AF04E5064
:10733800E1264F50E222E6CF50F0E5CF51F051C0A0
:1073480050F0516A5050DF6E20EE1EF05950D92689
:107358005A50DA2210EE0AF04E50E1264F50E2223F
:10736800E6CF50F0E6CF51F0E6CF52F0E6CF53F03B
:10737800110E05D0D8905332523251325032E82E85
:10738800F9D75050DF6E20EE1FF05950D9265A50C9
:10739800DA2210EE0AF04E50E1264F50E222E6CFF4
:1073A80050F0E6CF51F0E6CF52F0E6CF53F0190E89
:1073B80005D0D8905332523251325032E82EF9D794
:1073C8005050DF6E59C00BF05AC00CF020EE0EF092
:1073D8004E50D9264F50DA22DECF0DF0DECF0EF018
:1073E800DECF0FF0DECF10F017EC54F0556A566A76
:1073F800210E576E460E586E20EE16F05950D926BB
:107408005A50DA22DF6A20EE17F05950D9265A501E
:10741800DA2256C0DFFF20EE18F05950D9265A500C
:10742800DA2257C0DFFF20EE19F05950D9265A50FA
:10743800DA2258C0DFFF20EE12F05950D9265A50F0
:10744800DA22DF6A20EE13F05950D9265A50DA2290
:10745800DF6A20EE04F04E50D9264F50DA22DF0EB4
:10746800DF164EC0D9FF4FC0DAFF10EE04F0DE5031
:10747800E126DD50E222010EE76E4EC0D9FF4FC073
:10748800DAFFDECF43F0DDCF44F0AFEC2DF0546EE1
:107498005450120089800001FD6BF6EC3FF0CAC021
:1074A800B4F1CBC0B5F10101B451B51105E0B4C1D7
:1074B800EAF0B5C1EBF01200726AAC6BAD6BAE6B63
:1074C800AF6BB36B010EB26FB86BD4D0B66BB76B42
:1074D8001CD00EEC57F00B500C1013E0B80E0B6ECE
:1074E800010E0C6EC0EC4EF00101B16F000E72245B
:1074F800D96EDA6A030EDA22B1C1DFFF722AB64BFF
:10750800B72B0101B8AB81AC04D0B7BFE2D7B70540
:10751800E0E3B6C1ECF0B7C1EDF0000E0001EDBF3D
:10752800FF0EEE6FEF6FEC510101AC270001ED513A
:107538000101AD230001EE510101AE230001EF511D
:107548000101AF237350140D0F0EF324D96E010EF1
:10755800F420DA6EDE50AC5DDE50AD59DE50AE5927
:10756800DE50AF5902E3B26BB36BB8AB02D0B26B6B
:10757800B36B81BC02D0B26BB36BB7BF02D0B70597
:1075880019E2000E72240B6E0C6A030E0C22FF0E19
:107598007224D96EDA6A020EDA22DF500D6E0E6A94
:1075A800725000080F6E000ED8A0E82A0108106E6D
:1075B8000DEC44F00101AA513CE073503AE17350DC
:1075C800140D070EF324D96E010EF420DA6E84C16F
:1075D800F1F085C1F2F086C1F3F00001F06B000E06
:1075E800F025F46F010EF121F56F000EF221F66F10
:1075F800000EF321F76FDE50F4191BE1DE50F51988
:1076080018E1DE50F61915E1DE50F71912E101C351
:10761800BCF103C3BBF105C3BAF107C3B9F1B9C1E2
:107628000EF0BAC10FF0BBC110F0BCC111F014ECE0
:1076380053F0B5EC51F0E1510101B06FB0511AE0CF
:10764800010E0001FD6F7350140D130EF324D96E53
:10765800010EF420DA6E7350140D130EF324E16E4C
:10766800010EF420E26EE7500409DF6EFDC0EAF077
:10767800EB6B1200B251B31101E028D782A403D0FA
:10768800010E0001FD6F89900001EA6BEB6B12009F
:10769800736A736A030E736401D0E9D0735003E10F
:1076A8005A6A5B6A03D05B6A010E5A6E7350140DF6
:1076B800130EF324D96E010EF420DA6EDF6A7350CC
:1076C800140D000EF324D96E010EF420DA6EDF6A71
:1076D8007350140D070EF324D96E010EF420DA6EE0
:1076E800DE6ADE6ADE6ADD6A0D0E5A02F3CFA6F0A4
:1076F800F4CFA7F05B02F3500001A727E30EA625FD
:10770800D96E020EA721DA6EDF50A86FA8C0A9F0C3
:10771800AA6BAB6BAC6BABC0ACF0AAC0ABF0A9C0AA
:10772800AAF0A96B0D0E5A02F3CFADF0F4CFAEF06C
:107738005B02F350AE27E20EAD25D96E020EAE21E4
:10774800DA6EDF50AF6FAFC0B0F0B16BB26BB36B36
:10775800B1C0B3F0B0C0B2F0B16BB06B0D0E5A024D
:10776800F3CFB4F0F4CFB5F05B02F350B527E10ED8
:10777800B425D96E020EB521DA6EDF50B66FB6C0E9
:10778800B7F0B86BB96BBA6BB7C0BAF0B96BB86B76
:10779800B76B0D0E5A02F3CFBBF0F4CFBCF05B020F
:1077A800F350BC27E00EBB25D96E020EBC21DA6E61
:1077B800DF50B725BD6F000EB821BE6F000EB9218E
:1077C800BF6F000EBA21C06FB051BD25C16FB15156
:1077D800BE21C26FB251BF21C36FB351C021C46F64
:1077E800A951C125C56FAA51C221C66FAB51C3218A
:1077F800C76FAC51C421C86F7350140D0B0EF3241E
:10780800D96E010EF420DA6EC5C0DEFFC6C0DEFFF9
:10781800C7C0DEFFC8C0DEFFA30E806FFB0E816FFE
:1078280073C082F0836B7350140D0B0EF324D96E62
:10783800010EF420DA6EDECF84F0DECF85F0DECFE5
:1078480086F0DECF87F07350140D0B0EF324D96E3B
:10785800010EF420DA6EDECF88F0DECF89F0DECFBD
:107868008AF0DECF8BF0D3EC56F0732A13D70101E0
:107878009C6B0001FE6B01019B6B6B6A6C6A020ECC
:107888000001FD6F01019A6F8990020CF783340E95
:107898000B6E0A0E0C6E0E6A0D6A010E106E0F6AE0
:1078A8000DEC44F02AEE34F073C0DFFFFF0EE8CF92
:1078B80035FA7350140D130EF324D96E010EF4200B
:1078C800DA6EDFA403D0010EE8CF38FA7350140D36
:1078D800130EF324D96E010EF420DA6EDFA003D064
:1078E800020EE8CF3AFA7350140D130EF324D96E32
:1078F800010EF420DA6EDFA203D0020EE8CF3AFAC6
:107908007350140D130EF324D96E010EF420DA6EA1
:10791800DFA603D0800EE8CF39FA82A403D0080E80
:10792800E8CF3AFA626A636AC30E0001806FFB0E01
:10793800816FCFCF82F0836BCECF84F0856B62C02E
:1079480086F063C087F0360E6224D96E0A0E632073
:10795800DA6EDF50886F896BD3EC56F0000E622424
:10796800D96E020E6320DA6EDF1C616E360E622459
:10797800D96E0A0E6320DA6E360E6224E16E0A0EA4
:107988006320E26EE7506114DF6E5C0E0001806FC9
:10799800FF0E816F360E6224D96E0A0E6320DA6EEE
:1079A800DF50826F836BD3EC56F0624A632A63BE62
:1079B800BBD7635003E1070E625CB6E37350140D46
:1079C800130EF324D96E010EF420DA6EDF50000195
:1079D800FD6F7350140D010EF324D96E010EF420BF
:1079E800DA6EDF50606E60C03FFA7350140D020EFD
:1079F800F324D96E010EF420DA6EDF50606E60C099
:107A080040FA7350140D030EF324D96E010EF420BE
:107A1800DA6EDF50606E60C041FA7350140D040EC8
:107A2800F324D96E010EF420DA6EDF50606E60C068
:107A380042FA7350140D050EF324D96E010EF4208A
:107A4800DA6EDF50606E60C043FA7350140D060E94
:107A5800F324D96E010EF420DA6EDF50606E60C038
:107A680044FA5B6A140E5A6E3DEC3DF0F793899028
:107A780012000101A56B6D6A6E6A938693809382EA
:107A88009384938895688A908A928A948A98010E3A
:107A9800A46F898E89A4A46BF2981A0EE82EFED7DB
:107AA80000D007D0FC0E0001806FFF0E816FD3EC71
:107AB80056F081A8F7D7BBD081A881AA17D06EBE8F
:107AC80015D06E5002E16D0411E395689380280E7D
:107AD8000001806FFD0E816F6DC082F06EC083F073
:107AE800D3EC56F0630E0101A56FA7D0100E806F7E
:107AF800270E816F826B836B84D081B281A410D0F2
:107B08008007000E815B825B835B802906E1812907
:107B180004E1822902E18329D8A489D0620E67D0C2
:107B2800010E65D0020E63D05C685D685AC05EF0D5
:107B38005BC05FF05C505E265D505F226D505E1842
:107B480005E16E505F1802E1F7B3939A340E6D2485
:107B5800D96E0A0E6E20DA6EDF1C8C6E6D4A6E2AA4
:107B6800956A030E1ED0100E806F270E816F826BF0
:107B7800836B5DD081B20DD08007000E815B825B84
:107B8800835B802908E1812906E1822904E18329B0
:107B980002E1040EA56F81A24AD0040E28D093906A
:107BA800050EA56FE0D7938481B40DD08007000E31
:107BB800815B825B835B802908E1812906E1822958
:107BC80004E1832902E1060EA56F81A430D0060ED8
:107BD8000ED0938A938095685A506D5C6E50800AD7
:107BE8005C6E5B50800A5C589BE3630E0101A56FD5
:107BF8001ED09D0E0001806FFF0E816FD3EC56F0F2
:107C0800F4D7A5515C6E5D6A5D5011E15C5001E1ED
:107C180074D7010A87E0030A87E0010AABE0070A84
:107C2800BEE0010AC0E0030AD4E0640AE2E0630EA1
:107C38000101A51902E081BC3FD7F292F288A46B3A
:107C48009380938293849388938A9568899E6DC064
:107C58005AF06EC05BF0120081A605D01C0E000120
:107C6800A66FFE0E04D0B80E0001A66FFF0EA76F18
:107C780081AA04D01C0EA86FFE0E03D0B30EA86F05
:107C8800FF0EA96F81A804D01C0EAA6FFE0E03D0A8
:107C9800180EAA6FFF0EAB6F81AE04D01C0EAC6F2E
:107CA800FE0E03D0BD0EAC6FFF0EAD6F81AC04D0DD
:107CB8001C0EAE6FFE0E03D0AE0EAE6FFF0EAF6F92
:107CC80081A404D01C0EB06FFE0E03D0C70EB06F97
:107CD800FF0EB16F81A204D01C0EB26FFE0E03D04E
:107CE800CC0EB26FFF0EB36F81A004D01C0EB46F20
:107CF800FE0E03D0C20EB46FFF0EB56F83AE04D074
:107D08001C0EB66FFE0E03D0F60EB66FFF0EB76FE1
:107D180083AC04D01C0EB86FFE0E03D0F30EB86F00
:107D2800FF0EB96F83AA04D01C0EBA6FFE0E03D0E3
:107D3800F00EBA6FFF0EBB6F83A804D01C0EBC6F89
:107D4800FE0E03D0ED0EBC6FFF0EBD6F83A604D0F0
:107D58001C0EBE6FFE0E03D0EA0EBE6FFF0EBF6F85
:107D680083A404D01C0EC06FFE0E03D0E70EC06FB4
:107D7800FF0EC16F83A204D01C0EC26FFE0E03D08B
:107D8800E40EC26FFF0EC36F83A004D01C0EC46F35
:107D9800FE0E03D0E10EC46FFF0EC56FE00E806FBC
:107DA800FA0E816F831C826F836B81CF84F0856BA1
:107DB800C4C086F0C5C087F0C2C088F0C3C089F0CF
:107DC800C0C08AF0C1C08BF0BEC08CF0BFC08DF0BF
:107DD800BCC08EF0BDC08FF0BAC090F0BBC091F0AF
:107DE800B8C092F0B9C093F0B6C094F0B7C095F09F
:107DF800B4C096F0B5C097F0B2C098F0B3C099F08F
:107E0800B0C09AF0B1C09BF0AEC09CF0AFC09DF07E
:107E1800ACC09EF0ADC09FF0AAC0A0F0ABC0A1F06E
:107E2800A8C0A2F0A9C0A3F0A6C0A4F0A7C0A5F05E
:107E3800D3EF56F0636E0001CA5102E04CEC3BF000
:107E4800626A0001C95101E1B6D0040E631803E06B
:107E5800140E631809E101019B6B6B6A6C6A0001DF
:107E6800CA6B070EC96F070C3F0E631807E1FE6B5C
:107E780001019B6B0001C96BCA6B12005F0E63188E
:107E880007E101019C6B9B6B0001C96BCA6B120077
:107E98003F0E636406D05F0E636003D0400E631824
:107EA800F0E1400E631808E1010E01019C6F9B6B25
:107EB8000001C96BCA6B1200200E63180CE1010E99
:107EC800FE6F01019B6B7F0E0001806FFF0E816FBB
:107ED800D3EC56F0EDD7650E631809E1FE5107E0C3
:107EE8006B6A6C6A010E01019B6F8980E1D76E0E87
:107EF800631803E1020E01019B6F700E631807E11E
:107F080001019C5104E06B6A6C6A030E9B6F700E52
:107F1800631808E10001FE5105E089806B6A6C6A0C
:107F2800040E0CD0720E631846E10001FE5143E0C6
:107F380089801C0E6C6E2A0E6B6E050E01019B6FFC
:107F4800B7D7635016EC14F0626E47D0898063503F
:107F58008CEC4FF0626E01019B6B3FD08980340E30
:107F68000B6E0A0E0C6E0E6A0D6A010E106E0F6A09
:107F78000DEC44F00101F7832AEE34F0FDC0DFFF79
:107F88005B6A010E5A6E3DEC3DF0F793080EE2D79E
:107F98008990626A22D0080E631801E103D0090EA5
:107FA80063181BE18990626A0001FD6B01019B6BFC
:107FB8006B6A6C6A12D001019B51606E616A6150F4
:107FC8000CE160500AE0010ABCE0030ABFE0010AC4
:107FD800C5E0070ADDE0010ADEE062C0C9F0000181
:107FE800CA6B12007350140D070EF324D96E010EDC
:107FF800F420DA6EDECFDCF0DECFDDF0DECFDEF0AF
:10800800DECFDFF07350140D070EF324D96E010E86
:10801800F420DA6E7350140D0B0EF324E16E010E8A
:10802800F420E26EDE50E65CDE50E658DE50E6589C
:10803800DE50E65816E2010E0001FD6F7350140D74
:10804800130EF324D96E010EF420DA6E7350140D5A
:10805800130EF324E16E010EF420E26EE7500409DA
:10806800DF6E7350140D0F0EF324D96E010EF42039
:10807800DA6EDECFCCF0DECFCDF0DECFCEF0DECFC5
:10808800CFF07350140D070EF324D96E010EF420AF
:10809800DA6EDECFD0F0DECFD1F0DECFD2F0DECF99
:1080A800D3F00001CC51D025D46FCD51D121D56F5B
:1080B800CE51D221D66FCF51D321D76F7350140D23
:1080C8000B0EF324D96E010EF420DA6ED451DE5C67
:1080D800D551DE58D651DE58D751DE5815E2010E7B
:1080E800FD6F7350140D130EF324D96E010EF42096
:1080F800DA6E7350140D130EF324E16E010EF420A2
:10810800E26EE7500409DF6EFD6B7350200D080E18
:10811800F324A36F020EF420A46FDCC0A5F0DDC029
:10812800A6F0DEC0A7F0DFC0A8F077EC0EF0E06F95
:10813800E05115E0010EFD6F7350140D130EF3247A
:10814800D96E010EF420DA6E7350140D130EF32459
:10815800E16E010EF420E26EE7500409DF6EFDC007
:10816800CAF0CB6B12001B6E1B5001E0010C74A20D
:1081780002D074501200000E97EC56F00A0E266ECC
:1081880003D001EC57F026062650FBE1236A000EC7
:10819800146A156A166A176AEBEC54F0E80601E0EF
:1081A80097D0AA0E146E010E156E166A176A080E7D
:1081B800EBEC54F0E80651E1266A26501C0FD96E04
:1081C800DA6A01EC57F0DF6E262A030E2664F5D72B
:1081D8001E047EE1AA0E1F187BE1030E256EE80E31
:1081E800246E15D0146A156A166A400E176EA90E09
:1081F800EBEC54F000090EE00B0E1A6E620EE82E3E
:10820800FED71A2EFCD700D02406D8A02506245065
:108218002510E8E1245025105BE0146A156A166AF7
:10822800176A3A0EEBEC54F0000952E1266A265020
:108238001C0FD96EDA6A01EC57F0DF6E262A030E9E
:108248002664F5D71CBC03D0216A040E02D0216A2B
:108258000C0E206E20C023F03BD0146A156A166AF3
:10826800176AA90EEBEC54F01A6E020E1A6003D0CE
:10827800236EA90E02D0010E236E226E030E256E08
:10828800E80E246E14D0146A156A166A176A22500A
:10829800EBEC54F000090EE00B0E1A6E620EE82E9D
:1082A800FED71A2EFCD700D02406D8A025062450C5
:1082B8002510E9E1245025100AE0146A020E156E13
:1082C800166A176A100EEBEC54F0000901E0236AF5
:1082D80023C070F013EC57F0235001E14AD7749093
:1082E80048D7BEC0F6FFBFC0F7FF000EF86E0F0EEE
:1082F800F76403D00800F55005D0F6CFE9FFF7CFB3
:10830800EAFFEF502F0A13E0BEC0F6FFBFC0F7FF29
:10831800000EF86E0F0EF76403D00800F55005D074
:10832800F6CFE9FFF7CFEAFFEF505C0A03E100015F
:10833800BE4BBF2B000120EE06F0BC51D926BD5123
:10834800DA22DE6ADE6ADE6ADD6ABEC0F6FFBFC018
:10835800F7FF000EF86E0F0EF76403D00800F55013
:1083680005D0F6CFE9FFF7CFEAFFEF506A6E200E8F
:108378006A6012D0BCC062F0BDC063F0656A646A0E
:108388006CEC33F0C36F20EE12F0BC51D926BD510E
:10839800DA22DE6ADD6A5DD0BCC013F0BDC014F01D
:1083A800BE0E156EBDEC30F00001C36FC35151E134
:1083B800BCC0B6F0BDC0B7F0B9EC49F0C36F20EE51
:1083C80014F0BC51D926BD51DA2210EE0BF0DE5064
:1083D800E126DD50E222E750C26FC35108E0040EE7
:1083E800C31937E1C2B535D0050EC36F32D0C2B557
:1083F80030D020EE12F0BC51D926BD51DA22DECFA2
:10840800C0F0DDCFC1F020EE0BF0C051D926C1512C
:10841800DA22DFA8E9D7BCC0D9FFBDC0DAFFDECFBA
:108428000BF0DDCF0CF0C0C00DF0C1C00EF00DECAC
:108438004CF0000120EE06F0BC51D926BD51DA22DD
:108448000BC0DEFF0CC0DEFF0DC0DEFF0EC0DEFF7E
:10845800A3D7C35112000600D9CF05F0DACF06F032
:10846800F2A01CD081BC02D08994899281A802D044
:1084780089A20FD09380939424EE04F0010EDBBE02
:1084880007D0000EDE5C020EDE5802E3939201D0A4
:10849800938281B889B201D09384F290F2B281B00C
:1084A80079D081B889B29392831C086E811C076EBB
:1084B80004C409F005C40AF00ABE03D0020E0A5C1F
:1084C8002BE2094A0A2A09C004F40AC005F402C4C6
:1084D80009F003C40AF0060E0924D96E040E0A2016
:1084E800DA6E08C0DFFF060E0924D96E060E0A20D0
:1084F800DA6E07C0DFFF094A0A2A0168010E026E18
:1085080009C003F00AC004F0015003160250041613
:1085180003C002F404C003F481B889B2938493843D
:1085280081A0FED781A802D089A202D0939401D05D
:10853800938424EE04F0010EDBBE05D0000EDE5C51
:10854800020EDE5803E20101A45102E0939201D029
:10855800938207A81ED00BD0898202D0898405D0C7
:10856800899417D089A215D08994899212D008507D
:10857800016E026A02500DE10150040AF3E0100A8C
:10858800F1E0340AE9E01F0AF0E07F0AE7E01F0A99
:10859800E7E0F29206C0DAFF05C0D9FF7592110034
:1085A800326A20EE04F02450D9262550DA22DF5012
:1085B80001E197D020EE2AF02450D9262550DA225E
:1085C800DECF35F0DECF36F0DECF37F0DECF38F055
:1085D8002E0E24241A6E000E25201B6E35C01CF0AA
:1085E80036C01DF037C01EF038C01FF0216A010EDA
:1085F800206E20EE01F02450D9262550DA22DF50D3
:10860800DAEC48F0000903E0010E326E6AD020EE81
:1086180004F02450D9262550DA22DF6A20EE16F01D
:108628002450D9262550DA2210EE1EF02450E126D7
:108638002550E222E6CF2AF0E6CF2BF0E6CF2CF049
:10864800E6CF2DF02A50355C2E6E2B5036582F6E03
:108658002C503758306E2D503858316EDE502E5C05
:10866800DE502F58DE503058DE5031583AE220EEB6
:1086780003F02450D9262550DA22DF50336E346AAD
:10868800345003E1020E335C2CE320EE16F0245044
:10869800D9262550DA22DE503526DE503622DE5025
:1086A8003722DD5038222E0E24241A6E000E252083
:1086B8001B6E35C01CF036C01DF037C01EF038C028
:1086C8001FF0216A010E206E20EE01F02450D926F9
:1086D8002550DA22DF50DAEC48F03306D8A0340609
:1086E800CFD7325012002F6C696664617461302EE6
:1086F80062696E20002F6C696664617461312E6254
:10870800696E20002F6C696664617461322E62693B
:108718006E20002F6C696664617461332E62696E25
:1087280020002F6C696664617461342E62696E2062
:10873800002F6C696664617461352E62696E200071
:108748002F6C696664617461362E62696E20002F31
:108758006C696664617461372E62696E20002F6CE3
:10876800696664617461382E62696E20002F6C69D5
:108778006664617461392E62696E20002F6C6966C7
:1087880064617461612E62696E20002F6C69666491
:10879800617461622E62696E20002F6C6966646183
:1087A8007461632E62696E20002F6C69666461745F
:1087B80061642E62696E20002F6C69666461746161
:1087C800652E62696E20002F6C696664617461664B
:1087D8002E62696E2000000000000000000000000A
:1087E8000000000000000000000000000000000081
:1087F8000000000000000000000000000000000071
:108808000000000000000000000000000000000060
:1088180000000BC015F00CC016F00F50101001E14D
:10882800120015C0D9FF16C0DAFF0DC0DFFF0F50C8
:108838001524116E10501620126EFF0E1124D96ED9
:10884800FF0E1220DA6E0DC0DFFF105004E1030E98
:108858000F5C01E2120020EE01F01550D9261650E7
:10886800DA220DC0DFFF20EE02F01550D92616508F
:10887800DA220DC0DFFF0F501524116E105016209C
:10888800126EFE0E1124D96EFF0E1220DA6E0DC084
:10889800DFFF0F501524116E10501620126EFD0EBA
:1088A8001124D96EFF0E1220DA6E0DC0DFFF1050B2
:1088B80004E1070E0F5C01E2120020EE03F01550F0
:1088C800D9261650DA220DC0DFFF0F501524116E7D
:1088D80010501620126EFC0E1124D96EFF0E1220B5
:1088E800DA6E0DC0DFFF105004E1090E0F5C01E2E3
:1088F800120015C011F016C012F0111E121E114AF6
:10890800122A030E1114136E146A135015261450EC
:10891800162213500F5E1450105AFC0E0F160BD06F
:1089280015C0D9FF16C0DAFF0DC0DFFF0F06D8A0AB
:108938001006154A162A0F501010F2E11200000115
:10894800915190118F1103E1020E8E5D0FE320EE1D
:1089580012F08C51D9268D51DA22DE508E5DDE5010
:108968008F59DE509059DE50915902E3020E2CD0F7
:10897800966B6AD08CC044F08DC045F08EC046F02E
:108988008FC047F090C048F091C049F0C6EC1FF086
:1089980044C097F045C098F046C099F047C09AF097
:1089A80000019751981199119A115DE09705981156
:1089B80099119A11DBE0972909E1982907E199298A
:1089C80005E19A2903E1010E966F4DD08CC044F061
:1089D8008DC045F08EC046F08FC047F090C048F07B
:1089E80091C049F04A6A4B6A4C6A4D6A04EC19F026
:1089F800966F965138E120EE0EF08C51D9268D51A4
:108A0800DA22DE2806E1DE2804E1DE2802E1DE289B
:108A180013E020EE0EF08C51D9268D51DA22DE2A91
:108A2800000EDE22DE22DE2220EE05F08C51D92651
:108A38008D51DA22000EDB8097C08EF098C08FF03F
:108A480099C090F09AC091F020EE12F08C51D9267E
:108A58008D51DA22DE508E5DDE508F59DE509059EE
:108A6800DE50915987E396511200136814680B5031
:108A7800D96EDA6ADE50DE1001E181D00B50D96E72
:108A8800DA6ADECF17F0DDCF18F002D0174A182ABD
:108A980017C0F6FF18C0F7FF000EF86E0F0EF76448
:108AA80003D00800F55005D0F6CFE9FFF7CFEAFF6D
:108AB800EF500D6E200E0D6413D017C0F6FF18C0CE
:108AC800F7FF000EF86E0F0EF76403D00800F5509C
:108AD80005D0F6CFE9FFF7CFEAFFEF503A0AD6E123
:108AE80017C0F6FF18C0F7FF000EF86E0F0EF764F8
:108AF80003D00800F55005D0F6CFE9FFF7CFEAFF1D
:108B0800EF503A0A41E10B50D96EDA6ADECF11F024
:108B1800DDCF12F011C0F6FF12C0F7FF000EF86E9D
:108B28000F0EF76403D00800F55005D0F6CFE9FF23
:108B3800F7CFEAFFEF500D6ED00E0D24156E166AB2
:108B4800FF0E1622114A122A165019E10A0E155C58
:108B580016E21750111813E11850121810E11550A9
:108B680016100DE115C013F016C014F0174A182A94
:108B78000B50D96EDA6A17C0DEFF18C0DDFF13C0CC
:108B88000BF014C00CF01200136A146AF8D789802D
:108B9800B96BBA6B46EC50F05AC0BBF15BC0BCF184
:108BA800040E0101BC5D07E3000EBB25B96FFC0E86
:108BB800BC21BA6F04D0BBC1B9F1BCC1BAF1AA518A
:108BC80039E073500C0D540EF324D96E010EF420C5
:108BD800DA6E84C1B1F185C1B2F186C1B3F1B06B6F
:108BE800000EB025B46F010EB121B56F000EB22191
:108BF800B66F000EB321B76FDE50B4191BE1DE501B
:108C0800B51918E1DE50B61915E1DE50B71912E1B1
:108C180001C3C0F103C3BFF105C3BEF107C3BDF172
:108C2800BDC10EF0BEC10FF0BFC110F0C0C111F040
:108C380014EC53F082B418D07350200D080EF324AE
:108C48000001A36F020EF420A46F000EA56F030E9F
:108C5800A66F010EA86FA76BB90EA96F010EAA6FB8
:108C680007EC0BF00101B86F0101B8510AE0F10EF1
:108C78000001806FFD0E816FB8C182F0836BD3EC69
:108C880056F000EC28F0A86B8990800E0001806FE8
:108C9800FD0E816FCFCF82F0836BCECF84F0856BD2
:108CA800D3EF56F0020E0D5E000E0E5A0F5A105AF0
:108CB80020EE12F00B50D9260C50DA22FE0EDE24DC
:108CC800116EFF0EDE20126EFF0EDE20136EFF0EF9
:108CD800DE20146E11500D5C12500E5813500F58B0
:108CE8001450105805E30B6A0C6A0D6A0E6A1200DC
:108CF80020EE26F00B50D9260C50DA22DECF11F0E8
:108D0800DECF12F0DECF13F0DECF14F020EE02F04B
:108D18000B50D9260C50DA22DF50156E15C016F00C
:108D2800176A186A196A16500D02F3CF1AF0F4CFB1
:108D38001BF01C6A1D6A0E02F3501B26F4501C22FD
:108D4800000E1D2217500D02F3501B26F4501C2252
:108D5800000E1D2216500F02F3501C26F4501D223F
:108D680017500E02F3501C26F4501D2218500D0205
:108D7800F3501C26F4501D2210501602F3501D26E5
:108D880017500F02F3501D2618500E02F3501D26DF
:108D980019500D02F3501D2611501A240B6E125053
:108DA8001B200C6E13501C200D6E14501D200E6ECF
:108DB8001200F8C15CF070D049EC56F05C6EF819FE
:108DC80078E0150E5B6E4B0E5A6EBE0EE82EFED77F
:108DD8005A2EFCD75B2EFAD700D06BD012EC52F08B
:108DE8005D6E5D5066E05DB06F2A5DB26F060F0E76
:108DF8006F16000E0B6EC00EB0EC53F05CEC56F024
:108E0800000E0B6EC00EB0EC53F06F500F0D340E09
:108E1800F3240F6E0C0EF420106ECEEC4FF00D0EF6
:108E28005B6E2D0E5A6ED80EE82EFED75A2EFCD742
:108E38005B2EFAD75DA43DD00C6A0B6A6FC00DF0AB
:108E480096EC54F0150E0001806FFD0E816F6FC017
:108E580082F0836BD3EC56F06FC05CF0000E0B6EA3
:108E6800800EB0EC53F05CEC56F0000E0B6E800EEA
:108E7800B0EC53F06F500F0D340EF3240F6E0C0E40
:108E8800F420106ECEEC4FF0000E0B6EC00EB0EC5E
:108E980053F05CEC56F00DD00101A0515A6E5B6A9C
:108EA8005B5007E15A50010A87E0030A85E0010A8E
:108EB80095E05C5012001F6A206A186A196A01D08E
:108EC800122A010E1E6E1250D96EDA6A200EDE18B2
:108ED80013E0F70E146E15681250D96EDA6ADF5077
:108EE800166E176A1450162615501722175003E1EC
:108EF800050E165C01E31E6A1EC01AF01B6A1A50A2
:108F08001B1006E0DDD7196A010E186E122A25D04B
:108F18001250D96EDA6ADF50146E156A15501DE1C9
:108F280014502B0AF3E0060AEEE017D00A0E1F02CF
:108F3800F3CF14F0F4CF15F02002F3501526125099
:108F4800D96EDA6ADF50145E000E155A300E1424FA
:108F58001F6E000E1520206ED9D7D00E146E15681E
:108F68001250D96EDA6ADF50166E176A1450162638
:108F780015501722175005E10A0E165C02E2010E81
:108F880001D0000E1C6E1D6A1C501D10CFE1185038
:108F980019100DE11FC014F020C015F0141E151E85
:108FA800144A152A14C012F015C013F012001FC07D
:108FB80012F020C013F01200A86B8980000E0B6E0F
:108FC800030E0C6E0E6AF60E0D6E010E106E0F6A11
:108FD8000DEC44F0950E0001806FFE0E816FD3EC0E
:108FE80056F00101B66BB76B2E0EDDEC56F082B46D
:108FF80018D07350200D080EF3240001A36F020E41
:10900800F420A46F000EA56F030EA66F010EA86FC3
:10901800A76BB20EA96F010EAA6F07EC0BF0010146
:10902800B46F0101B4510AE0780E0001806FFF0EA1
:10903800816FB4C182F0836BD3EF56F00EEC57F01A
:109048000B500C1026E0B50E0B6E010E0C6EC0EC2A
:109058004EF00101B16FB551100B5A6E000E5B6EE8
:10906800B151ADEC1DF05AC0B8F15BC0B9F1040EB6
:109078000101B819B91102E19EEC55F0020EB819B8
:10908800B91102E18BEC53F0B805B91102E161ECBA
:109098001BF00101B64BB72B600EB65D040EB75935
:1090A800A3E3270E0001806FFF0E816FD3EC56F00B
:1090B80089901200BA6B898075D046EC50F05AC07E
:1090C800B8F15BC0B9F1040E0101B95D03E3010E0B
:1090D800BA6F03D0BDC1BBF1BC6B82B418D073505A
:1090E800200D080EF3240001A36F020EF420A46FD4
:1090F800000EA56F030EA66F010EA86FA76BBB0E1F
:10910800A96F010EAA6F07EC0BF00101BD6FBD51ED
:109118000AE0F10E0001806FFD0E816FBDC182F083
:10912800836BD3EC56F00101AA5139E073500C0D52
:10913800540EF324D96E010EF420DA6E84C1B1F115
:1091480085C1B2F186C1B3F1B06B000EB025B46F22
:10915800010EB121B56F000EB221B66F000EB3211A
:10916800B76FDE50B4191BE1DE50B51918E1DE50B7
:10917800B61915E1DE50B71912E101C3C1F103C3F5
:10918800C0F105C3BFF107C3BEF1BEC10EF0BFC138
:109198000FF0C0C110F0C1C111F014EC53F000EC95
:1091A80028F0A86BBA5189E089901200236E2350E9
:1091B800D8A4040C2050211001E1040C74B0030C55
:1091C80074B4020C70B608D0090ED8901C361D363F
:1091D8001E361F36E82EF9D7200421101AE11CC0CC
:1091E80014F01DC015F01EC016F01FC017F0180EA1
:1091F800EBEC54F0000945E11AC00DF01BC00EF06D
:10920800FE0E0F6EC0EC52F000093BE0206A216AA6
:1092180038D070C022F0060E221609E020C014F0E3
:1092280021C015F0166A176A970EEBEC54F01CC0B3
:1092380014F01DC015F01EC016F01FC017F0190E4F
:10924800EBEC54F000091DE11AC00DF01BC00EF044
:10925800FC0E0F6EC0EC52F0000908E0020E1B264F
:109268002006D8A0210620502110EEE10D6A0E6AD2
:10927800FD0E0F6EC0EC52F0000903E1216A010EE9
:10928800206E13EC57F020502110D8A4010C000CCC
:109298000F0EC16E969496929690929A090E106E41
:1092A8001E0E0F6EE40EE82EFED70F2EFCD7102EE2
:1092B800FAD700D0090E106E1E0E0F6EE40EE82EBF
:1092C800FED70F2EFCD7102EFAD700D0D00E0F6E77
:1092D800CA0EE82EFED70F2EFCD7000E0B6E300EEE
:1092E800B0EC53F0150E0F6EC60EE82EFED70F2EFB
:1092F800FCD700D0000E0B6E300EB0EC53F0000E11
:109308000B6E300EB0EC53F0000E0B6E390EB0EC55
:1093180053F0000E0B6E140EB0EC53F0000E0B6EF3
:10932800560EB0EC53F0000E0B6E6D0EB0EC53F011
:10933800000E0B6E700EB0EC53F0000E0B6E0C0EA0
:10934800B0EC53F0000E0B6E060EB0EC53F0000EAE
:109358000B6E010EB0EC53F0680E0F6EE40EE82EA3
:10936800FED70F2EFCD700D01200B6C062F0B7C0EF
:1093780063F0656A646A6CEC33F0BB6FBB5102E062
:10938800BB511200B6C0D9FFB7C0DAFFDECF39F043
:10939800DDCF3AF020EE0EF0B651D926B751DA22D9
:1093A800DECF3BF0DECF3CF0DECF3DF0DECF3EF04F
:1093B80006EC4DF00001BB6FBB51E2E120EE12F06C
:1093C800B651D926B751DA22DECFB9F0DDCFBAF0DF
:1093D800B9C0D9FFBAC0DAFFDF50B86FB85103E19E
:1093E800040EBB6FCDD720EE0BF0B951D926BA5178
:1093F800DA22DFB616D0B9C00BF0BAC00CF020EEF6
:1094080014F0B651D926B751DA22DECF0DF0DDCFF0
:109418000EF0106A0B0E0F6EE5EC51F00B500C10AD
:10942800AFE0B6C0A3F0B7C0A4F0A66BA56BFBEC89
:1094380029F00001BB6FBB51A3E1A4D7B6C062F00D
:10944800B7C063F0656A646A6CEC33F0BF6FBF51F4
:1094580057E1BD6BBE6BB6C0D9FFB7C0DAFFDECF30
:1094680039F0DDCF3AF020EE0EF0B651D926B751DB
:10947800DA22DECF3BF0DECF3CF0DECF3DF0DECFB0
:109488003EF006EC4DF00001BF6FBF5139E120EE10
:1094980012F0B651D926B751DA22DECFBAF0DDCFB5
:1094A800BBF0BAC0D9FFBBC0DAFFE50EDE1810E08A
:1094B80020EE12F0B651D926B751DA22DECFBAF033
:1094C800DDCFBBF0BAC0D9FFBBC0DAFFDF5009E17E
:1094D800BD4BBE2BB851BD1906E1B951BE1910E0FC
:1094E80002D0BD6BBE6BB6C0A3F0B7C0A4F0A66B2C
:1094F800010EA56FFBEC29F00001BF6FBF51ABE077
:10950800040EBF1902E1070EBF6FBF511200EE0E25
:10951800F66E860EF76E000EF86E0CEE34F011EE55
:109528002CF00900F5CFEEFFE550E150FAE1E250EA
:10953800F8E1CC0EF66EA60EF76E000EF86E02EE8F
:10954800B2F010EE4AF00900F5CFEEFFE550E15019
:10955800FAE14B0EF66EAE0EF76E000EF86E0900CD
:10956800F5CFFAF14A0EF66EAE0EF76E000EF86EF3
:109578000900F5CF74F004EE00F018EE34F0EE6A4E
:10958800E550E150FCE1E250FAE103EE00F011EEA3
:1095980000F0EE6AE550E150FCE1E250FAE102EE3B
:1095A80000F0B20EEE6AE806FDE101EE00F0AC0E46
:1095B800EE6AE806FDE10001FF6BFE6BFD6B00EE55
:1095C8006BF0090EEE6AE806FDE175907592000EE3
:1095D800F86E000149EF07F00101A96B716A966BFB
:1095E800976B020EA86F8990A76BA66B736A030E20
:1095F800736401D049D073500C0D530EF324D96E07
:10960800010EF420DA6EDF6A73500C0D520EF3244B
:10961800D96E010EF420DA6EDF6A73500C0D500E0D
:10962800F324D96E010EF420DA6EDE6ADD6A735017
:109638000C0D540EF324D96E010EF420DA6EDE6A96
:10964800DE6ADE6ADD6A73500C0D5B0EF324D96E98
:10965800010EF420DA6E100EDF6E73500C0D5A0EE8
:10966800F324D96E010EF420DA6E020EDF6E735009
:109678000C0D580EF324D96E010EF420DA6E240E68
:10968800DE6EDD6A732AB3D7100E01015B6F020E1E
:109698005A6F596B240E586F736A1200C0C0B6F027
:1096A800C1C0B7F0B96B010EB86F22EC4AF06A6E10
:1096B8006A5053E1C0C0D9FFC1C0DAFFDECF39F02C
:1096C800DDCF3AF020EE0EF0C051D926C151DA2292
:1096D800DECF3BF0DECF3CF0DECF3DF0DECF3EF01C
:1096E80006EC4DF06A6E6A5038E1000120EE12F087
:1096F800C051D926C151DA22DECF0BF0DDCF0CF0F4
:109708000E6A0D6A106A200E0F6E21EC56F00001E9
:1097180020EE12F0C051D926C151DA22DECF0BF06B
:10972800DDCF0CF020EE14F0C051D926C151DA2259
:10973800DECF0DF0DDCF0EF0106A0B0E0F6E59EC78
:1097480054F0C0C0D9FFC1C0DAFF10EE04F0DE50FB
:10975800E126DD50E222010EE76E6A501200F7831F
:10976800735028E1340E0B6E0A0E0C6EF20E0D6E5D
:10977800020E0E6E106A050E0F6EF6EC53F0390EDF
:109788000B6E0A0E0C6EB20E0D6E020E0E6E106A85
:10979800130E0F6EF6EC53F04C0E0B6E0A0E0C6E99
:1097A800D80E0D6E020E0E6E106A0D0E0F6EF6ECD0
:1097B80053F027D0340E0B6E0A0E0C6EF70E0D6E9A
:1097C800020E0E6E106A050E0F6EF6EC53F0390E8F
:1097D8000B6E0A0E0C6EC50E0D6E020E0E6E106A22
:1097E800130E0F6EF6EC53F04C0E0B6E0A0E0C6E49
:1097F800E50E0D6E020E0E6E106A0D0E0F6EF6EC73
:1098080053F05B6A250E5A6E3DEC3DF0F793899054
:1098180012001A0E0D240F6E000E0E20106E0F2867
:10982800D96E000E1020DA6EDF50126E116A1A0E11
:109838000D24D96E000E0E20DA6EDF50111211C001
:1098480017F012C018F0196A1A6A0BC0D9FF0CC0B9
:10985800DAFF030EDE1829E1140E0D240F6E000E38
:109868000E20106E0F28D96E000E1020DA6EDF5011
:10987800126E116A140E0D24D96E000E0E20DA6EC7
:10988800DF501110136E1250146E156A166A14C048
:1098980016F013C015F0146A136A135017121450F7
:1098A80018121550191216501A1217C00BF018C0BA
:1098B8000CF019C00DF01AC00EF012008980000ECD
:1098C8000B6E030E0C6E0E6AF60E0D6E010E106E08
:1098D8000F6A0DEC44F0950E0001806FFE0E816F4B
:1098E800D3EC56F00001CA6BCB6B2E0EDDEC56F0B4
:1098F80082B416D07350200D080EF3240001A36F14
:10990800020EF420A46F000EA56F030EA66F010EC1
:10991800A86FA76BC70EA96FAA6B07EC0BF0C96FEE
:109928000001C95109E0780E806FFF0E816FC9C030
:1099380082F0836BD3EF56F0CA4BCB2BCBBFD5D776
:10994800CB5103E1640ECA5DD0E3270E806FFF0E92
:10995800816FD3EC56F0899089900001FD6B12005D
:10996800226E2250D8A4040C2050211001E1040CCE
:1099780074B0030C70B608D0090ED8901C361D368A
:109988001E361F36E82EF9D7215006E1020E205C5C
:1099980003E2246A110E02D0246A120E236E23C039
:1099A80025F01CC014F01DC015F01EC016F01FC015
:1099B80017F02550EBEC54F000091DE11AC00BF02C
:1099C8001BC00CF0020E0E6E0D6A3FEC52F000093F
:1099D80008E0020E1B262006D8A0210620502110E0
:1099E800EDE1120E251807E1146A156A166A176A5E
:1099F8000C0EEBEC54F013EC57F020502110D8A4C7
:109A0800010C000C436A20EE2AF03950D9263A504E
:109A1800DA223B50DE1809E13C50DE1806E13D50E1
:109A2800DE1803E13E50DE1839E039C024F03AC0B0
:109A380025F0D4EC42F0436E435030E12E0E392429
:109A48001A6E000E3A201B6E3BC01CF03CC01DF085
:109A58003DC01EF03EC01FF0216A010E206E20EEB0
:109A680001F03950D9263A50DA22DF50B4EC4CF0E4
:109A7800000906E03B683C683D683E68010E436E9D
:109A880020EE2AF03950D9263A50DA223BC0DEFFC0
:109A98003CC0DEFF3DC0DEFF3EC0DEFF435012008B
:109AA800D4C0DAF0D5C0DBF0DA0E0B6E39EC45F035
:109AB8000BC0DCF00CC0DDF00001DDBF0B0CD89052
:109AC800DC35D96EDD35DA6E940ED926010EDA2230
:109AD800DECFD8F0DDCFD9F0D851D91105E0D8C004
:109AE800D9FFD9C0DAFFDF6AD251D31105E0D2C05D
:109AF800D9FFD3C0DAFFDF6AD890DC35D96EDD35FF
:109B0800DA6E940ED926010EDA22D2C0DEFFD3C057
:109B1800DDFFD251D311D8B4000CD60501E0000CFA
:109B2800D20E666E676AD40E686E696A09EC00F038
:109B3800D76FD751120003D00B4A0C2A0D2A0D50AB
:109B4800D96EDA6ADF500E6E0BC0F6FF0CC0F7FF55
:109B5800000EF86E0F0EF76403D00800F55005D01C
:109B6800F6CFE9FFF7CFEAFFEF500E1813E10BC06D
:109B7800F6FF0CC0F7FF000EF86E0F0EF76403D067
:109B88000800F55005D0F6CFE9FFF7CFEAFFEF5010
:109B98000009D2E10BC0F6FF0CC0F7FF000EF86E0B
:109BA8000F0EF76403D00800F55005D0F6CFE9FF93
:109BB800F7CFEAFFEF500E6E0D50D96EDA6ADF501C
:109BC8000E5C0B6E0C6AD8A00C0612007350140DB4
:109BD800070EF324D96E010EF420DA6E000EDE248F
:109BE800CA6F010EDE20CB6F000EDE20CC6F000E98
:109BF800DE20CD6F7350140D070EF324D96E010EBD
:109C0800F420DA6ECAC0DEFFCBC0DEFFCCC0DEFFB8
:109C1800CDC0DEFF7350140D070EF324D96E010E6C
:109C2800F420DA6EDECFCEF0DDCFCFF07350200D0A
:109C3800080EF324A36F020EF420A46FCEC0A5F083
:109C4800CFC0A6F0A76BA86B77EC0EF0D06FD05101
:109C580003E0010EFD6F010CFD6B12000BC012F04A
:109C68000CC013F00DC014F00EC015F00F06D8A0EC
:109C780010060F280CE110280AE10B6A0C6A120082
:109C8800124A132A144A152A0F06D8A0100612C021
:109C9800F6FF13C0F7FF0800F55015E014C0D9FF10
:109CA80015C0DAFFDF500FE00F5010100CE014C0A1
:109CB800D9FF15C0DAFF12C0F6FF13C0F7FFDE5058
:109CC8000900F518DDE012C0F6FF13C0F7FF080021
:109CD800F5CF11F014C0D9FF15C0DAFFDF50115CC1
:109CE8000B6E0C6AD8A00C0612000CC012F00DC046
:109CF80013F012501310D8B4090C12C0D9FF13C0B6
:109D0800DAFFDE50DE10D8B4090C12C0D9FF13C038
:109D1800DAFFDECF0EF0DDCF0FF00EC0D9FF0FC097
:109D2800DAFFDF50D8B4090C20EE02F01250D92621
:109D38001350DA2212C0E1FF13C0E2FF00EE06F072
:109D4800E650E926E550EA22DE50EE1813E1DE502F
:109D5800EE18D8A4090C12C0D9FF13C0DAFF10EE10
:109D680001F0DE50E126DD50E222E75008EC57F022
:109D78000E6E0EB0090C000C24EE04F0DE50DE105E
:109D8800FBE000C413F001C414F0060E1324D96ECE
:109D9800040E1420DA6EDF50116E060E1324D96EED
:109DA800060E1420DA6EDF50126E134A142A0D685C
:109DB800010E0E6E13C00FF014C010F00D500F16E8
:109DC8000E5010160FC000F410C001F4F29E24EEDD
:109DD80004F0DE06000EDD5AF28E0BC0D9FF0CC06F
:109DE800DAFF12C0DFFF24EE04F0010EDBBE05D05F
:109DF800000EDE5C020EDE5802E289B29382115038
:109E080012000E5002E00E5003E10C50C9EF56F05C
:109E18000E50D96EDA6A040ED926DE50DE1014E030
:109E28000E50D96EDA6A040ED9260E50E16EE26A37
:109E3800020EE126DE50E65CE650800A136EDE5024
:109E4800800A1358D8B012000E50D96EDA6A020E82
:109E5800D926DECF0FF0DDCF10F00E50D96EDA6ABA
:109E6800DECF11F0DDCF12F00F501124D96E105053
:109E78001220DA6E0CC0DFFF0E50D96EDA6A020EBD
:109E8800D926DE2A000EDD22000C0B500F02F3CF7C
:109E980013F0F4CF14F0156A166A0B501002F35041
:109EA8001426F4501522000E16220C500F02F350FF
:109EB8001426F4501522000E16220B501102F350EE
:109EC8001526F45016220C501002F3501526F450A3
:109ED80016220D500F02F3501526F4501622125078
:109EE8000B02F35016260C501102F35016260D5093
:109EF8001002F35016260E500F02F350162613C008
:109F08000BF014C00CF015C00DF016C00EF01200C6
:109F1800010E0001806FFE0E816F6BC082F06CC075
:109F280083F0D3EC56F010D0030E0AD0050E5C6E09
:109F38006B6A6C6A2DD00A0E03D0010E01D0020E96
:109F48005C6E26D05C6A24D06BC05AF06CC05BF0A3
:109F58005B5009E0020A0DE00E0A0FE0010A11E069
:109F68002A0A13E0EFD75A500A0ADEE01E0ADEE09A
:109F7800E9D75A50BC0AE3E0E5D75A501C0ADBE09F
:109F8800E1D75A50AC0AD9E0DDD75A500F0ADAE1C6
:109F98005C5012000B0E116E620EE82EFED7112EC9
:109FA800FCD700D020D00B0E116E620EE82EFED723
:109FB800112EFCD700D0010E0B6E0FC0F6FF10C09B
:109FC800F7FF000EF86E0F0EF76403D00800F55087
:109FD80005D0F6CFE9FFF7CFEAFFEF50B0EC53F02A
:109FE8000F4A102AD7D70FC0F6FF10C0F7FF000E90
:109FF800F86E0F0EF76403D00800F55005D0F6CFC1
:10A00800E9FFF7CFEAFFEF500009CDE11200136A2C
:10A01800146A156A166A0F5010101110121029E0F0
:10A02800010E176E06D0D8900F361036113612363C
:10A03800172A12AEF8D7D8901336143615361636B6
:10A048000F500B5C10500C5811500D5812500E58F0
:10A0580009E30F500B5E10500C5A11500D5A125054
:10A068000E5A1380D8901232113210320F32172E36
:10A07800E2D713C00BF014C00CF015C00DF016C0D9
:10A088000EF012005D6A5E6A726A5F6A2ED00EEC8C
:10A0980057F00B500C101EE05F0E0B6E0C6AC0ECF4
:10A0A8004EF05C6E5FA80BD0120E0001806FFF0EA1
:10A0B800816F5CC082F0836BD3EC56F00BD0000E3E
:10A0C8007224D96EDA6A030EDA225CC0DFFF722AC4
:10A0D8005D4A5E2A5FAA07D0000E5D245A6E040E00
:10A0E8005E205B6E120081AC02D05E04D0E35DC0DE
:10A0F8005AF05EC05BF01200136E0C0E131807E0E6
:10A1080013EC57F0B1EC56F0000901E1FF0C1350C5
:10A118004009F0EC56F01050F0EC56F00F50F0EC0F
:10A1280056F00E50F0EC56F00D50F0EC56F0010ED3
:10A13800126E135002E1950E126E080E131802E10A
:10A14800870E126E1250F0EC56F00C0E131802E146
:10A1580001EC57F00A0E126E01EC57F0116E11AEB9
:10A1680002D0122EF9D71150120089800001AF6B6E
:10A17800B06BB16BB26B7350200D080EF324626E96
:10A18800020EF420636E340E646E0A0E656E010EC4
:10A19800676E666AB30E686E696A61EC11F0000159
:10A1A800AE6F0101F793B3C05AF0B4C05BF03DEC59
:10A1B8003DF05AC0ACF05BC0ADF00001AC51AF2728
:10A1C800AD51B023000EB123B2230101A86B8990D1
:10A1D800120007EC55F0CC0E8AEC56F0660E8AECAD
:10A1E80056F06DEC56F0156E155005E10F6A106AC1
:10A1F800116A126A1200136A146A1350150FD96E85
:10A20800DA6A6DEC56F0DF6E134A142A14BEF5D7DD
:10A21800145003E1040E135CF0E3185017101610E5
:10A2280003E1060E155CE2E315C00FF016C010F04E
:10A2380017C011F018C012F01200736A030E73648D
:10A2480001D02AD073500C0D530EF324D96E010E91
:10A25800F420DA6EDF6A73500C0D520EF324D96EB7
:10A26800010EF420DA6EDF6A73500C0D500EF324E1
:10A27800D96E010EF420DA6EDE6ADD6A73500C0DB9
:10A28800540EF324D96E010EF420DA6EDE6ADE6A0B
:10A29800DE6ADD6A732AD2D7736A8990A86B1200C6
:10A2A8000F5010101110121023E0010E136E06D07B
:10A2B800D8900F36103611361236132A12AEF8D748
:10A2C8000F500B5C10500C5811500D5812500E586E
:10A2D80008E30F500B5E10500C5A11500D5A1250D3
:10A2E8000E5AD8901232113210320F32132EE8D78C
:10A2F8000BC00BF00CC00CF00DC00DF00EC00EF032
:10A3080012000B6A0C6A7350140D070EF324D96EF1
:10A31800010EF420DA6EDE6ADE6ADE6ADD6A7350E8
:10A32800140D130EF324D96E010EF420DA6EDF6AD1
:10A338007350140D0F0EF324D96E010EF420DA6E4B
:10A34800DE6ADE6ADE6ADD6A0B4A0C2A0CBEDBD7DF
:10A358000C5003E1040E0B5CD6E389900001FD6B01
:10A368001200F6EC3FF0CAC0E5F0CBC0E6F0E551CC
:10A37800E61105E0E5C0E1F0E6C0E2F0120082B4C3
:10A3880015D07350200D080EF324A36F020EF4208D
:10A39800A46F000EA56F030EA66F010EA86FA76B22
:10A3A800E30EA96FAA6B07EC0BF0E76FE75104E027
:10A3B800E7C0E1F0E26B1200EAEC4DF0E16BE26B12
:10A3C80012000BC012F00CC013F00DC014F00EC038
:10A3D80015F0166A176A0F06D8A010060F2802E1B2
:10A3E800102817E012C0D9FF13C0DAFF124A132A47
:10A3F800DF50116E14C0D9FF15C0DAFF144A152AB0
:10A40800DF50115C166E176AD8A017061650171081
:10A41800E2E016C00BF017C00CF01200010E0B6E34
:10A428000C6A92868D828D8400D000D000D000D036
:10A438008D9400D000D000D000D00D6A0E6A80A69E
:10A4480002D00B500C12D8900B368D9000D000D053
:10A4580000D000D08D8000D000D000D000D08D90EA
:10A468000D4A0E2A0EBEEBD70E5003E1030E0D5C0B
:10A47800E6E30C501200070E106ED00E0F6E0CD0D3
:10A4880001EC57F0116E11280AE1A00E00D0E82E59
:10A49800FDD70F06D8A010060F501010F1E1FE0EE0
:10A4A800111801E0000C01EC57F00BC0D9FF0CC0EB
:10A4B800DAFFDF6E0B4A0C2A0D06D8A00E060D50E7
:10A4C8000E10F1E101EC57F001EC57F0010C0BC054
:10A4D80011F00CC012F013D00F06D8A010060DC052
:10A4E800D9FF0EC0DAFF0D4A0E2A11C0E1FF12C0D3
:10A4F800E2FF114A122ADFCFE7FFE7500BE00F50C7
:10A50800101008E0E9D711C0D9FF12C0DAFFDF6ADE
:10A51800114A122A0F06D8A010060F28F4E11028B5
:10A52800F2E112008C6A8A6A956893680101A46B4B
:10A53800726A89928994906B916B09D0000E90256C
:10A54800D96E030E9121DA6EDF6A904B912B91BF81
:10A55800F5D79105F3E3906B916B09D0340E9025F4
:10A56800D96E0A0E9121DA6EDF6A904B912B91BF5A
:10A57800F5D79105F3E312006FEC55F0000901E1FE
:10A58800000C0F50F0EC56F0FD0E0F181EE0020EF6
:10A59800116E106A0DC0D9FF0EC0DAFFDF50F0EC63
:10A5A80056F00D4A0E2A1006D8A0110610501110A8
:10A5B800F1E101EC57F001EC57F001EC57F0126EA5
:10A5C80012501F0B050A01E0000C010C15D00CC03D
:10A5D800F6FF0DC0F7FF000EF86E0F0EF76403D0FC
:10A5E8000800F55005D0F6CFE9FFF7CFEAFFEF50A6
:10A5F800DDEC56F00C4A0D2A0CC0F6FF0DC0F7FF33
:10A60800000EF86E0F0EF76403D00800F55005D061
:10A61800F6CFE9FFF7CFEAFFEF500009D8E11200C3
:10A628000EC012F00FC013F010C014F011C015F0D6
:10A6380007EC55F0CC0E8AEC56F0990E8AEC56F0E1
:10A648000C0E8AEC56F0166A176A1650120FD96E5D
:10A65800DA6ADF508AEC56F0164A172A17BEF5D781
:10A66800175002E007EF55F0040E165CEEE307EF13
:10A6780055F05B6E990E5C6EFA0E5D6E5A6A0AD0E2
:10A688005CC0F6FF5DC0F7FF5C4A5D2A0800F55024
:10A69800F7E15A2A5B505A1807E05CC0F6FF5DC024
:10A6A800F7FF0800F550ECE1870E0001806FFE0E01
:10A6B800816F5BC082F0836B5CC084F05DC085F005
:10A6C800D3EF56F001091220010001001700002DF8
:10A6D800119420D00F000101091220010001001778
:10A6E80000002D119420D00F000100004F01000F31
:10A6F8000000000009FF0000004F01000F000000EB
:10A708000009FF00800102E805800102E805898050
:10A71800F7832AEE34F0A6C1DFFF000EE8CF35FA42
:10A728000D0EE8CF36FA000EE8CF37FA82A403D030
:10A73800600EE8CF37FA82A406D036CA60F0200E41
:10A74800601260C036FA5B6A040E5A6E3DEC3DF04A
:10A75800F793A66B899012000C6E8D9200D000D0F2
:10A7680000D000D00BB002D08D9401D08D84000EA3
:10A778000E6E010E0D6E0CAE02D0898A01D0899A38
:10A78800D8900C368D908D808D900D4A0E2A0EBE75
:10A79800F2D70E5003E1090E0D5CEDE38D82120035
:10A7A8009F0E136E146811C015F012C016F01350E6
:10A7B800152614501622165005E11A0E155C02E2F1
:10A7C800010E01D0000E176E186A1750181005E018
:10A7D8005F0E1114116E126A120011C011F012C02E
:10A7E80012F012000DC013F00EC014F00BC011F0DF
:10A7F8000CC012F010D013C0D9FF14C0DAFFDF501C
:10A80800156E134A142A11C0D9FF12C0DAFF15C0F9
:10A81800DFFF114A122A0F06D8A010060F28EBE115
:10A828001028E9E1120020EE1AF00B50D9260C503E
:10A83800DA220DC0DFFF20EE1BF00B50D9260C509A
:10A84800DA220EC0DFFF20EE14F00B50D9260C5090
:10A85800DA220FC0DFFF20EE15F00B50D9260C507E
:10A86800DA221050DF6E12000BC00DF00CC00EF093
:10A8780002D00B4A0C2A0BC0F6FF0CC0F7FF000EE3
:10A88800F86E0F0EF76403D00800F55005D0F6CF28
:10A89800E9FFF7CFEAFFEF500009EBE10D500B5C41
:10A8A8000B6E0E500C580C6E12000BC011F00CC041
:10A8B80012F00DC013F00EC014F00ED013C0D9FF63
:10A8C80014C0DAFF11C0E1FF12C0E2FFDFCFE7FFDB
:10A8D800134A142A114A122A0F06D8A010060F2864
:10A8E800EDE11028EBE112000B6E0B500EE01AECB4
:10A8F80057F0200EE82EFED71DEC57F0CC0E00D0F6
:10A90800E82EFDD700D000D012001AEC57F0C00E88
:10A9180000D0E82EFDD71DEC57F0350EE82EFED7F7
:10A9280000F01200000EF2BE010E0E6E0C50030B6A
:10A93800AA6E0BC0A9FF0DC0A8FFA69EA69CA68460
:10A94800F29E550EA76EAA0EA76EA682A6B2FED7D5
:10A95800A6940EB002D0F29E01D0F28E120002D060
:10A968000B4A0C2A0BC0F6FF0CC0F7FF0800F55085
:10A9780009E00BC0F6FF0CC0F7FF0800F5500D18F2
:10A988000E10EEE10BC0F6FF0CC0F7FF0800F55003
:10A998000B6E0C6A12005E0E626E5AC063F05BC0EA
:10A9A80064F0656A666A676A686A630E546E5CC0BA
:10A9B80055F05DC056F0620E576EEFEC23F065500F
:10A9C8005A24D96E66505B20DA6EDF6A000C186E66
:10A9D80018AE0ED0189E0D6A0E6A0F6A106A370EEE
:10A9E80080EC50F0196E010E196402D01950120053
:10A9F80014C00DF015C00EF016C00FF017C010F0FF
:10AA0800185080EF50F01AEC57F00A0E0C6EF80E42
:10AA1800E82EFED70C2EFCD700D01DEC57F0E00E28
:10AA280000D0E82EFDD7E7EC56F0090E0C6E840E28
:10AA3800E82EFED70C2EFCD71DEF57F0010E116E35
:10AA4800200E0B180C1011E0F70E0D6E0E680BC0DF
:10AA58000FF00CC010F00D500F260E5010221050A1
:10AA680003E1050E0F5C01E3116A11C00BF00C6ADB
:10AA780012005BC04EF05CC04FF045EC39F05D6EE3
:10AA88005D500FE15BC00CF05CC00DF079EC4EF04E
:10AA98005D6E5D5006E15BC0D9FF5CC0DAFFDE6A1F
:10AAA800DD6A5D5012009F0E0D6E0E68200E0B10B1
:10AAB8000F6E000E0C10106E0D500F260E50102247
:10AAC800105005E11A0E0F5C02E2010E01D0000ED3
:10AAD8000B6E0C6A1200130E0C6E880E0B6E0BD0E8
:10AAE80001EC57F0FF0A0AE0A00E00D0E82EFDD7CF
:10AAF8000B06D8A00C060B500C10F2E10B500C10F2
:10AB0800D8A4010C000C186A196A09D017C00CF0F7
:10AB18000D6A16C00EF005EC4FF0184A192A1850A5
:10AB28001424D96E19501520DA6EDF50176E17509D
:10AB3800EDE11200340E0B6E0A0E0C6E0E6A0D6AF1
:10AB4800010E106E0F6A0DEC44F02AEE34F0A8C125
:10AB5800DFFF5B6A010E5A6E3DEC3DF0A86B1200F8
:10AB6800340E0B6E0A0E0C6E0E6A0D6A010E106E14
:10AB78000F6A0DEC44F0010EE8CF34FA0101F783B7
:10AB88005B6A5A6E3DEC3DF0F79312009F0E0D6E16
:10AB98000E680BC00FF00CC010F00D500F260E50B1
:10ABA8001022105005E11A0E0F5C02E2010E01D0CE
:10ABB800000E0B6E0C6A1200BF0E0D6E0E680BC0F5
:10ABC8000FF00CC010F00D500F260E501022105030
:10ABD80005E11A0E0F5C02E2010E01D0000E0B6EA9
:10ABE8000C6A1200D00E0D6E0E680BC00FF00CC070
:10ABF80010F00D500F260E501022105005E10A0ECD
:10AC08000F5C02E2010E01D0000E0B6E0C6A1200FE
:10AC1800B886AC84B898440EAF6EB06AAC98AB8E68
:10AC2800AB88AB9A9D989D9AD08E9F8AF28EAC90F5
:10AC3800AB9CAC9AAC8A9D9112000BC011F00CC071
:10AC480012F008D011C0D9FF12C0DAFF0DC0DFFF23
:10AC5800114A122A0F06D8A010060F28F3E110286F
:10AC6800F1E112001AEC57F0200EE82EFED71DEC89
:10AC780057F0300EE82EFED7E7EC56F00C6EB00E0B
:10AC880000D0E82EFDD70C501200070E966E8450A7
:10AC9800070B0B6E928A80AA02D0080E0B26020EB2
:10ACA8000101A01903E10B1C0F0B0B6E0B501200D6
:10ACB800106A100E0F6E05D0010E0B6E200EB0EC50
:10ACC80053F00F06D8A010060F28F6E11028F4E17B
:10ACD80012000D6A0E6AD8900D3236EC56F0000953
:10ACE80001E00D8E0E2A070E0E64F5D70D501200E6
:10ACF800000EE8CF00F4E8CF01F4E8CF02F4E8CF83
:10AD080003F4E8CF04F4E8CF05F4000C0C6E0D6AE8
:10AD18000C50010B78EC54F0D8900C320D2A070E29
:10AD28000D64F6D7070C0B6E0B5007E0C66A010ED0
:10AD3800C66E400EC76EC68A400CC66A020EF8D7A9
:10AD4800C2900F0EC16E070EB46E4F0EC86E946A95
:10AD5800948894829482826A120022EC57F001EC63
:10AD680057F06FEC55F0000901E0010C13EC57F0B7
:10AD7800000C0C50030BAA6E0BC0A9FFA69EA69C44
:10AD8800A68000F000F0A85012000B6E03D024EC4F
:10AD980057F004009EA8FBD70BC0ADFF1200820E2F
:10ADA800596E80C018F081C019F0590E1A6EFAEF6A
:10ADB80025F00B6E03D024EC57F004009EA8FBD7B7
:10ADC8000BC0ADFF1200928880A803D0010E0B6E55
:10ADD80001D00B6A0B5012000B6E0BC0C9FFC7B035
:10ADE800FED7C7A0FED7C95012000B6E02D08988C3
:10ADF80089980B060B28FBE11200C968C7B0FED77B
:10AE0800C7A0FED7C95012000B6E0B5001E0010C11
:10AE18007450120004C40BF005C40CF0120020ECAE
:10AE280057F001EF57F08990A86B12008998929813
:10AE38001200899892881200828012008290120073
:04AE4800120001E70C
:10FA9800004F4B004449534B5F455252004E4F5460
:10FAA8005F5245414459004E4F5F46494C45004E10
:10FAB8004F545F4F50454E4544004E4F545F454E9E
:10FAC80041424C4544004E4F5F46494C455F5359AF
:10FAD8005354454D000020000D0A2025325820259A
:10FAE8003258202532732025327320253273202581
:10FAF8003273202532732025327320253273202556
:10FB0800327320253473202534732025347320253F
:10FB1800347320253473202534732025347320252D
:10FB2800347320000D0A48504469736B204D6B20D4
:10FB38004949202831384634363230292025732067
:10FB48002573202573205374617274696E672E2E95
:10FB58002E0D0A000D0A5365656B2065727220250B
:10FB680064203E2025642C202564203E2025642C1A
:10FB7800202564203E202564000D0A52642075204B
:10FB880025642072746E2025642C202564206279F7
:10FB980074657320726561640D0A000D0A4D617801
:10FBA80020566563746F72206469736B2025642026
:10FBB800256C642028256C582920000D0A25303230
:10FBC80058253032582053533830783A537461747A
:10FBD80075735B25645D20255820000D0A44736BFE
:10FBE80073656C2069732025642C206E756D6265C1
:10FBF800722069732025642000466F756E64206149
:10FC08006E205254432066696C6520617420255823
:10FC18000D0A004C6F6F6B696E6720666F7220610A
:10FC28006E205254432066696C650D0A0046696E61
:10FC38006446696C65206661696C656420736561FA
:10FC48007263680D0A000D0A4469736B2073656C52
:10FC5800656374206E756D626572202564000D0AF7
:10FC68005365656B20746F20256C64206661696C30
:10FC78006564202564000D0A4F70656E696E672003
:10FC88006578697374696E6720257320000D0A47CB
:10FC98006F7420256C7520202D207265736574742F
:10FCA800696E67005365656B696E6720746F2073B2
:10FCB8006563746F722025580D0A0046696E6446A4
:10FCC800696C65206661696C656420726561640DA4
:10FCD8000A000D0A4469736B205374617475733A92
:10FCE8002025582C20000D0A57616974696E672019
:10FCF800666F72206361726420000D0A46696C6544
:10FD0800202573206973206F70656E20000D0A57D7
:10FD1800726F7465206469736B6E6F3A2025640096
:10FD28002041544E206173736572746564203120DC
:10FD38002564000D0A4F70656E696E67206E6577E1
:10FD480020257320000D0A46696C65202558206916
:10FD58007320257320000D0A4469736B20255820F1
:10FD6800697320257320004E6F742061204C49462A
:10FD7800206469736B0D0A000D0A2530325825304E
:10FD88003258204578697420000D0A52656164690B
:10FD98006E67205254430D0A000D0A416D69676F62
:10FDA8002039313231440D0A000D0A53532F3830AF
:10FDB8002039313232440D0A000D0A44736B7365E1
:10FDC8006C20697320256420000D0A526561642047
:10FDD8002564206279746573000D0A487374206283
:10FDE8007974657332202564000D0A577269746549
:10FDF800206661696C202564000D0A53533830650C
:10FE080078656320256420000D0A4F70656E696E61
:10FE1800672025732020000D0A44656275672069F4
:10FE28007320256420000D0A50726F746F20697367
:10FE380020256420000D0A5265616420636F6E6698
:10FE4800696720000D0A46696C656E616D6520253D
:10FE5800732000566563746F722069732025580DEE
:10FE68000A00222A2B2C3A3B3C3D3E3F5B5D7C7FBF
:10FE7800000D0A56616C75653A2025580D0A007206
:10FE8800633D25752046525F25730D0A000D0A460D
:10FE98006F726D617474696E6720000D0A4E6F2071
:10FEA80063617264202564002F6C69666461746103
:10FEB8002E62696E000D0A25732025582025580DDD
:10FEC8000A002A2A20566572696679202A2A000DB6
:10FED8000A73627974657331202564000D0A4D6FC9
:10FEE800756E74696E6720004A616E203131203268
:10FEF800303231004C6F6164696E672E2E2E0068B7
:10FF0800706469736B2E636667002025582077201C
:10FF180041544E20005B535251206F66665D004687
:10FF28006D742065786974200031393A31313A317D
:10FF380030005B2532582025645D005B5352512008
:10FF48006F6E5D0048504469736B20004E6F2063EC
:10FF5800617264002D3E202558200044534B5345C0
:10FF68004C004E414D452558004449534B255800F7
:10FF780072633D256420005B4D4C415D0044454261
:10FF880055470050524F544F005265616479002024
:10FF980025303258007B4552527D000D0A44534AA1
:10FFA80000302E3136004946432000454F49200095
:10FFB80052454E2000535251200044415620004ED5
:10FFC800444143004E5246440052544300202558B1
:10FFD8000025325800207C20004430004431004481
:10FFE800320044330044340044350044360044377A
:07FFF800002563002B00004F
:020000040020DA
:08000000FFFFFFFFFFFFFFFF00
:020000040030CA
:0E000000FF06191EFF8181FF0FC00FE00F40A9
:00000001FF
